:1000000000400020B5620000F5620000F7620000C9
:1000100000000000000000000000000000000000E0
:10002000000000000000000000000000F962000075
:100030000000000000000000FB620000FD62000004
:10004000FF620000152E0000E96A0000FF62000058
:10005000FF62000000000000FF620000FF6200007D
:10006000FF6200002D650000FF620000FF620000DB
:10007000FF620000FF620000FF620000FF620000FC
:10008000FF6200008D6B0000FF620000FF62000055
:10009000FF620000FF620000FF620000FF620000DC
:1000A000FF620000FF62000000000000000000008E
:1000B0000000000000000000000000000000000040
:1000C000054B0648033310B51B1A062B03D9044B06
:1000D000002B00D0984710BD3802002038020020C5
:1000E000000000000648074910B5091A8910CB0F17
:1000F0005918491003D0044B002B00D0984710BD6D
:1001000038020020380200200000000010B5074C23
:100110002378002B09D1FFF7D3FF054B002B02D02A
:10012000044800E000BF0123237010BD3802002006
:100130000000000070AE0000094B10B5002B03D08A
:100140000849094800E000BF08480368002B02D1B5
:10015000FFF7C8FF10BD064B002BF9D09847F7E713
:10016000000000003C02002070AE000034020020BD
:1001700000000000164B002B00D1144B9D4640227E
:1001800092029A1A924600218B460F461348144A4F
:10019000121A08F004FC0F4B002B00D098470E4BAE
:1001A000002B00D098470020002104000D000D48CE
:1001B000002802D00C4800E000BF08F0ADFB200092
:1001C000290006F0A9FC08F081FBC04600000800E9
:1001D0000040002000000000000000003802002065
:1001E000E024002000000000000000000123034084
:1001F0000200181E04D1042A03D91068000900E087
:100200000020704710B50400FFF7F0FF0300002046
:1002100083420BD0013B9B00181DE2181279002A83
:1002200003D001338342F8D100E0180010BD012251
:10023000016810B5114201D0002903DA102000F046
:10024000E3F903E04910062001F032FF10BD016818
:1002500010B5CB0701D5002903DA102000F0D4F93E
:1002600006E04910033189100022052001F020FF2B
:1002700010BD70B50568AB0728D1042D26D90F2312
:100280002A6846681340062B09D12800FFF7AEFF05
:10029000012383421DDC9A00AE500133F9E7052BA0
:1002A00014D1F30703D4132000F0AEF912E0761056
:1002B000FF2EF8D82800FFF799FF2C1D230080009F
:1002C0002018984205D91E700133FAE70B2000F080
:1002D0009BF9002070BD70B50468E30701D41120BC
:1002E0002DE04568AB0729D1042D27D90F262B68AF
:1002F00064101E40062E0BD1002C04DD2800FFF7F1
:1003000075FF844201DD122019E0A400605918E055
:10031000331F012B12D82800FFF768FF8000042E3E
:1003200002D12800FFF76EFF002CECDDA042EADBD3
:1003300001232C19E0784000184302E00B2000F064
:1003400063F970BDF8B5012304681C4201D1112086
:100350002FE00325466835402AD1042E28D90F23E3
:100360003268641087681340062B0BD1002C04DD23
:100370003000FFF73BFF844201DD122019E0A400AA
:10038000A75113E0052B13D1002CF6DD3000FFF749
:100390002DFF80008442F0DC01231F4201D1132095
:1003A00007E07F10FF2FFAD83419E770280002E029
:1003B0000B2000F029F9F8BD006810B5830717D1AC
:1003C000042815D90F2302681340062B02D1FFF72A
:1003D0000DFF0BE0052B05D1FFF708FFC00001233F
:1003E000184308E0042B03D1FFF70CFF4000F6E7A9
:1003F0000B2000F009F910BD10B50324006804407B
:1004000006D1042804D90F2302681340042B01D01D
:100410000E2011E001F088FE0378233B5942594138
:1004200010224018210008F093FF80239B05C2187A
:10043000054B9A4203D9142000F0E6F802E00123AC
:100440004000184310BDC046FFFFFF3F10B5012418
:100450000368234202D04268224203D10D2000F0FB
:10046000D3F808E004495B1052101B070A401343FD
:1004700018684000204310BDFCFFFF0F01210368F6
:1004800010B50B4205D042680A4202D0806808428B
:1004900003D10D2000F0B8F808E005495B105210B8
:1004A0001B070A40401013431860002010BDC046CF
:1004B000FCFFFF0F012303400200181E01D0501063
:1004C00002E00D22014B1A707047C0465402002012
:1004D000012303400200181E04D1042A03D9106826
:1004E000000900E00020704770B50D000400FFF720
:1004F000EFFF86002800FFF7EBFF830000209E42FD
:100500000ED1231D9E1904351A009E4207D9297861
:100510001278013301358A42F6D0002000E0012034
:1005200070BD0000F0B585B00393019002912D4E8F
:100530002D4B002A02D002223270013A00251A60A7
:100540001B68F554019B9D424ADA029AAB00D058D1
:10055000254B1C68C8239B0037191C1B012318421C
:1005600002D04310214A1FE0214A002802D004286B
:1005700005D1204A2100380008F0D8FD18E00428F1
:1005800010D90F2302681340042B04D101F0CCFDD5
:10059000194A030008E0062B05D1FFF799FF174A17
:1005A000030001E00123164A2100380008F0BEFDD7
:1005B000300008F021FE039B0B4A002B01D1106094
:1005C0000CE0019B013B9D42F9DA0E4B9842F6DCB0
:1005D000431C1360202232540022F2540135B1E74B
:1005E00005B0F0BD600200205C0200201DA10000EB
:1005F000F0A00000F6A000004EA40000FBA0000048
:100600000CA100001F030000014B18700020704770
:100610005402002070B503F055FA094C0100251D65
:100620001F22280008F0EFFD280008F0E5FD042354
:1006300004308008000118432060200070BDC046CF
:1006400080050020C368F0B59E00836889B09E19BC
:100650000300183306930369069A9C00069B0290D8
:100660001D19436901939B00D3180393D74B1B7843
:10067000002B0FD17F223368D5491C1213409B00F9
:100680005B582F000436019233E0D04B1B78002BCF
:1006900027D03D00029BCD4C9B6821780193F21A34
:1006A000029B92109B7812021A43029B587802F028
:1006B00095FF0023029A23701370029B069A9B6891
:1006C000F61A0193029BB610DE60069BED1A029BA0
:1006D000AD101D61039B9B1A029A9B10536101F0A0
:1006E00034FC3368019A1C121340B94A9B009B5892
:1006F00004369F46029B587802F068FF0023029A56
:10070000137001F03DF9069B3D1DEA1AAF4BDB2A41
:1007100003DD1A223D001A70BCE71B783C60002BF9
:10072000B8D13368019A1C121340A94A9B009B5808
:100730002F000436DDE7069B3D1DEA1AA34BDB2A9A
:1007400003DD1A223D001A70A4E731681B78321DC0
:100750003960002B01D016009CE77368019A1C12C7
:1007600013409B4A9B009B582F000836C1E7069B0D
:100770003D1DEA1A954BDB2A03DD1A223D001A7053
:1007800088E7A4001B7834193C60002B82D13368C1
:10079000019A1C1213408E4A9B009B582F0004366E
:1007A000A7E7069B3D1DEA1A884BDB2A03DD1A22C8
:1007B0003D001A706EE7874AA400A2581B783A6081
:1007C000002B00D066E73368019A1C121340804A60
:1007D0009B009B582F0004368BE73D1F7D4B2A68FA
:1007E000A400E250794B1B78002B00D052E733680D
:1007F000019A1C121340764A9B009B582F00043626
:1008000077E7A3000493049A724B3D1FD058FFF77B
:1008100051FE04002868FFF74DFE241801206D4B9F
:100820006400049A0443D450684B1B78002B00D01A
:1008300030E73368019A1C121340654A9B009B58AD
:100840002F00043655E7069B3D1DEA1A5F4BDB2A55
:1008500003DD1A223D001A701CE703990698012255
:10086000814202D90A000C3A12681B783A60002BC8
:1008700000D00FE73368019A1C121340544A9B00C2
:100880009B582F00043634E7069B3D1DEA1A4F4B58
:10089000DB2A03DD1A223D001A70FBE6039A069953
:1008A0008A420AD913000C3B1B684B4A5B10A41800
:1008B000E41A039BA400E35802E018221A700023F4
:1008C0003B60424B1B78002B00D0E3E63368019A73
:1008D0001C1213403E4A9B009B582F00043608E729
:1008E000039B069A93420BD90C3B1B683A4A5B1058
:1008F000A4183D1FE41A2A68039BA400E25003E0F9
:1009000018223D00314B1A70304B1B78002B00D061
:10091000C0E63368019A1C1213402D4A9B009B5875
:100920002F000436E5E6039B069A93421FD92A4B13
:100930003D1FE318039C04930C3C2368049A5B104E
:10094000D31A039A9B009858FFF7B4FD07902868C4
:10095000FFF7B0FD2468049B64101C1B079BA400D8
:100960001F1801207F00039B0743E75003E0182274
:100970003D00164B1A70154B1B78002B00D089E6F2
:100980003368019A1C121340114A9B009B582F0098
:100990000436AEE6069B3D1DEA1A0C4BDB2A03DD4E
:1009A0001A223D001A7075E6039AA400A2581B781B
:1009B0003A60002B00D06DE63368019A1C12134098
:1009C000034A9B009B582F00043692E654020020F5
:1009D000F09E000050230020FDFFFF3F3D1F039BC2
:1009E0002A68A400E250D34B1B78002B00D051E6BC
:1009F0003368019A1C121340CF4A9B009B582F006A
:100A0000043676E6039BA4001C1923683D1F5B1087
:100A100028680493FFF74EFD049B1F180120C54B67
:100A20007F001B7807432760002B00D032E6336835
:100A3000019A1C121340C04A9B009B582F00043699
:100A400057E6069BA4003D1BBA4CAB420DD8237859
:100A5000002B00D01EE63368019A1C121340B64AE0
:100A60009B009B582F00043643E6B44801F0D2FAAD
:100A70002378002B00D00DE63368019A1C12134036
:100A8000AD4A9B009B582F00043632E6A300F618AF
:100A9000002C01DA00F074FFA64B1B78002B01D06C
:100AA0003D00F7E53368019A1C121340A24A9B00EF
:100AB0009B5804361DE63D1F2B68042B04D1A30070
:100AC000F618002C06DAF8E5002B03D00C22994B1F
:100AD0001A70DFE5974B1B78002B00D0DAE53368FE
:100AE000019A1C121340944A9B009B582F00043615
:100AF000FFE53D1F2B68002B04D1A300F618002C46
:100B000006DADAE5042B03D00C228A4B1A70C1E511
:100B1000884B1B78002B00D0BCE53368019A1C126F
:100B20001340854A9B009B582F000436E1E53A1F8D
:100B300013685B10013B002B07DD01215B00A40063
:100B40000B433D0036191360B7E57A4B15001B784F
:100B5000002B00D09EE5336801991C120B407649AA
:100B60009B005B5817000436C3E53A00069B0C3225
:100B7000D31ADB2B04DD1A226E4B3D001A7089E577
:100B8000FF2361005B000B4001210B433B60029B94
:100B900006989B6824120493F61A029BB6109B7861
:100BA00036021E43039B8E401B1A9B108B400B4347
:100BB000BB60029B0E437E609C70E4B2604BE4001D
:100BC0000299E35815008B605A490978002903D02F
:100BD00008331E0003925DE51E0001999B680C36E8
:100BE0001C120B4054499B005B580392170080E590
:100BF0003B1F1C68069A039B93422AD13D000A20A2
:100C0000E30716D4A3070DD1042C0BD90F232268B8
:100C10001340042B06D1200001F086FA08F0ECFA0C
:100C2000063006E00720042C03D0002C01D08020E1
:100C30008000643002F07AFA002801D1043E3CE5DD
:100C4000029B2100587802F0DBFC0023029A13700B
:100C500033E5039B03990C3B1B685B109B005B42D5
:100C60001A00CB180C3B1C600B00083B1B68083AB1
:100C70008D1802995A108A70D2B23149D2005B00A5
:100C800056589B0A029A9B009660F618039B069A98
:100C9000043B1B685B109B00D3180393254B1B7808
:100CA000002B00D0F6E43368019A1C121340224A4C
:100CB0009B009B582F0004361BE53B1F1868FFF76D
:100CC000F9FBA40004903D1B1E282ADC00280EDC42
:100CD000184B1B78002B00D0DCE43368019A1C12FF
:100CE0001340154A9B009B582F00043601E502F083
:100CF000CFFE049F033F3F1802F0CAFE114BC01BFA
:100D00009842F9D80B4B1B78002B00D0C2E4336813
:100D1000019A1C121340084A9B009B582F0004366E
:100D2000E7E40123029A137002F0B2FE049B0A3832
:100D3000C71834E054020020F09E000020A10000FB
:100D4000581B00209F8601003B1F1868FFF7B2FB6D
:100D5000A40004903D1B00280EDCD44B1B78002B14
:100D600000D097E43368019A1C121340D04A9B00CC
:100D70009B582F000436BCE4CE4B049A9A4203DD04
:100D80001D22CA4B1A7085E40123029A137002F0E7
:100D90007FFEFA23049F9B005F430A3F3F18029B9C
:100DA0005F608AE40023A5007D1B1A002000290053
:100DB000FFF7B8FBC04FC14C3968200002F06CFB54
:100DC0003968200002F023FCB84B1B78002B00D0C0
:100DD00060E43368019A1C121340B54A9B009B588B
:100DE0002F00043685E4B14BA4001B783D1B002B7B
:100DF00000D04FE43368019A1C121340AC4A9B00A8
:100E00009B582F00043674E402F0D6F901F09DF8E7
:100E10003B1F1868002823D1083B1868C30701D579
:100E2000401016E083070FD104280DD90F23026864
:100E30001340062B02D1FFF74BFB0AE0052B03D131
:100E4000FFF746FB800004E01922984B3D001A7022
:100E500020E43A0001214300083A0B43136001E00B
:100E600040100138002832DD012243001343391FAE
:100E70000B603B00083B1B681341181A3B000C3BFE
:100E80001B68134203D08018A400904015E0990716
:100E900017D1042B15D90F211D682940062906D129
:100EA00001308000C358039AA400A35010E0052924
:100EB00007D118180079A4004000039B1043E050AC
:100EC00006E01922794B3D001A70FFF7E3FB043668
:100ED000764B1B78002B02D03D00FFF7DBFB33681D
:100EE000019A1C121340724A9B009B580436FFF76C
:100EF00000FCA300069AFB189B1ADB2B02DC3D00CA
:100F0000012205E01A22694B3D001A70FFF7C2FB6F
:100F1000631E002C03DD2A601C000435F8E7634BD8
:100F20001B78002B01D0FFF7B5FB3368019A1C1228
:100F300013405F4A9B009B582F000436FFF7D9FBF4
:100F4000A3009C46F81A002C04DC1C22574B0025F9
:100F50001A7015E0002103685B1001258A00825891
:100F6000154003D10D22514B1A7009E052109342E3
:100F700000DD130001318C42EFDC01255B001D43D5
:100F800063460560FD1A494B04351B78002B01D0E0
:100F9000FFF780FB3368019A1C121340444A9B0000
:100FA0009B582F000436FFF7A4FBA3009C46F81AB9
:100FB000002C04DC1C223D4B00251A7015E000219A
:100FC00003685B1001258A008258154003D10D2269
:100FD000364B1A7009E05210934200DA13000131C7
:100FE0008C42EFDC01255B001D4363460560FD1A62
:100FF0002E4B04351B78002B01D0FFF74BFB3368D9
:10100000019A1C1213402A4A9B009B582F00043659
:10101000FFF76FFB3B00083B1868FFF74BFA3B1FDD
:1010200004901868FFF746FA049AA5007C1B002379
:10103000824200DA043323601C4B7D1B1B7804358D
:10104000002B01D0FFF726FB3368019A1C121340D6
:10105000174A9B009B582F000436FFF74AFBA3005A
:10106000FD1A04933B00083B1868FFF723FA3B1F67
:1010700004001868FFF71EFAE20FC317A04253419D
:101080009B002B60049BFD1A084B04351B78002B3A
:1010900001D0FFF7FFFA3368019A1C121340044A8B
:1010A0009B009B582F000436FFF723FB54020020BF
:1010B000F09E000080EE36005C02002060020020FE
:1010C0003B00083B18683B1F1968A300884202D107
:1010D000FB1A042222E004281ED90122104201D06A
:1010E000114219D10325284215D10F2302681A4055
:1010F000042A10D129420ED104290CD90A681340C0
:10110000042B08D1FFF7F0F9431E9841A5007D1B81
:101110008000286003E0A3000022FB1A1A60D84B6D
:10112000A4001B783D1B0435002B01D0FFF7B2FA59
:101130003368019A1C121340D24A9B009B582F001F
:101140000436FFF7D6FA3B00083B18683B1F1968C6
:10115000A300884202D1FB1A002223E004281FD9F1
:101160000122104201D011421AD10325284216D182
:101170000F2302681A40042A11D129420FD10429F1
:101180000DD90A681340042B09D1FFF7ADF903000C
:1011900058425841A5007D1B8000286003E0A30051
:1011A0000422FB1A1A60B64BA4001B783D1B0435C1
:1011B000002B01D0FFF76EFA3368019A1C1213401E
:1011C000B04A9B009B582F000436FFF792FAA30009
:1011D000FD1A04933B00083B1868FFF76BF93B1FAF
:1011E00004001868FFF766F9E217C30F8442534101
:1011F0009B002B60049BFD1AA14B04351B78002B30
:1012000001D0FFF747FA3368019A1C1213409D4A38
:101210009B009B582F000436FFF76BFA3B00083BFE
:101220001868FFF747F93B1F04901868FFF742F969
:10123000049AA5007C1B0023824200DD0433236056
:101240008F4B7D1B1B780435002B01D0FFF722FA52
:101250003368019A1C1213408A4A9B009B582F0046
:101260000436FFF746FA3B1F1B68854AA400042B8F
:1012700002D13B1B002103E0002B03D104213B1BC7
:10128000196001E00C23137013783D1B0435002B0B
:1012900001D0FFF7FFF93368019A1C121340794A15
:1012A0009B009B582F000436FFF723FAA3000493FA
:1012B000FC1A3B00083B1868FFF7FCF83B1F0500D1
:1012C0001868FFF7F7F82D180120049B6D000543FF
:1012D0002560FD1A6A4B04351B78002B01D0FFF7FF
:1012E000D9F93368019A1C121340664A9B009B5837
:1012F0002F000436FFF7FDF9A300FD1A04933B000D
:10130000083B1868FFF7D6F83B1F04001868FFF782
:10131000D1F8241A0120049B640004432C60FD1AB8
:10132000574B04351B78002B01D0FFF7B3F9336816
:10133000019A1C121340534A9B009B582F000436FD
:10134000FFF7D7F9A3000493FC1A3B00083B186889
:10135000FFF7B0F83B1F05001868FFF7ABF84543EF
:101360000120049B6D0005432560FD1A444B0435A4
:101370001B78002B01D0FFF78DF93368019A1C12FE
:101380001340404A9B009B582F000436FFF7B1F9E9
:101390003B00083B1868FFF78DF83B1F0490186866
:1013A000FFF788F80100049805F0BEFC0123A500B2
:1013B0007C1B250040001843314B20601B7804350E
:1013C000002B01D0FFF766F93368019A1C12134015
:1013D0002C4A9B009B582F000436FFF78AF93B00EC
:1013E000083B1868FFF766F83B1F04901868FFF782
:1013F00061F80100049805F07DFD0123A5007C1B28
:101400002500490019431E4B21601B780435002B31
:1014100001D0FFF73FF93368019A1C121340194AB3
:101420009B009B582F000436FFF763F93B1F186899
:10143000FFF740F8C317C018584001234000184375
:101440000F4BA4001B783D1B28600435002B01D0F6
:10145000FFF720F93368019A1C121340094A9B00D8
:101460009B582F000436FFF744F9A300FD1A079399
:101470002868012C08D1FFF71DF804900DE0C04644
:1014800054020020F09E0000FFF714F80400686882
:10149000FFF710F80130031B0493049B002B01DCC1
:1014A0000123049307F0F4FD049905F023FD0C19C2
:1014B0000121079B64000C432C60FD1AF84B043596
:1014C0001B78002B01D0FFF7E5F83368019A1C1256
:1014D0001340F44A9B009B582F000436FFF709F98C
:1014E000A4003D1B2800FEF787FFED4B28601B780A
:1014F0000435002B01D0FFF7CDF83368019A1C1298
:101500001340E84A9B009B582F000436FFF7F1F880
:10151000A300FD1A04933B00083B1868FEF7CAFFBE
:101520003B1F04001868FEF7C5FF04400120049B20
:10153000640004432C60FD1AD94B04351B78002B42
:1015400001D0FFF7A7F83368019A1C121340D54A5F
:101550009B009B582F000436FFF7CBF8A3000493A1
:10156000FC1A3B00083B1868FEF7A4FF3B1F050070
:101570001868FEF79FFF05430120049B6D0005439B
:101580002560FD1AC64B04351B78002B01D0FFF7F0
:1015900081F83368019A1C121340C24A9B009B5881
:1015A0002F000436FFF7A5F8A3000493FC1A3B00B4
:1015B000083B1868FEF77EFF3B1F05001868FEF722
:1015C00079FF45400120049B6D0005432560FD1A0D
:1015D000B34B04351B78002B01D0FFF75BF8336861
:1015E000019A1C121340AF4A9B009B582F000436EF
:1015F000FFF77FF83B1F1868FEF75CFFC04301232D
:1016000040001843A64BA4001B783D1B28600435FE
:10161000002B01D0FFF73EF83368019A1C121340EB
:10162000A04A9B009B582F000436FFF762F8A300E6
:10163000FD1A04933B00083B1868FEF73BFF3B1F75
:1016400004001868FEF736FF8440012364001C4341
:10165000049B2C60FD1A924B04351B78002B01D0A3
:10166000FFF718F83368019A1C1213408D4A9B004B
:101670009B582F000436FFF73CF8A300FD1A049393
:101680003B00083B1868FEF715FF3B1F0400186875
:10169000FEF710FF0441012364001C43049B2C60EF
:1016A000FD1A7F4B04351B78002B01D0FEF7F2FFAB
:1016B0003368019A1C1213407A4A9B009B582F00F2
:1016C0000436FFF716F83B000C3B1868FEF7F2FEF5
:1016D0003B00083B05001868FEF7ECFEE917020026
:1016E000C317280005F058FC3B1F049005911868AB
:1016F000FEF7E0FE02000498059905F001FC0123C5
:1017000040001843664BA4001B783D1B286004353D
:10171000002B01D0FEF7BEFF3368019A1C12134064
:10172000604A9B009B582F000436FEF7E2FFA4009E
:101730003D1B2800FEF77BFD594B28601B780435C4
:10174000002B01D0FEF7A6FF3368019A1C1213404C
:10175000544A9B009B582F000436FEF7CAFFA40092
:101760003D1B2800FEF773FD4D4B28601B780435A8
:10177000002B01D0FEF78EFF3368019A1C12134034
:10178000484A9B009B582F000436FEF7B2FFA40086
:101790003D1B2800FEF76DFD414B1B78002B01D04F
:1017A000FEF778FF3368019A1C1213403D4A9B00F4
:1017B0009B582F000436FEF79CFFA4003D1B280019
:1017C000FEF789FD364B28601B780435002B01D0CD
:1017D000FEF760FF3368019A1C121340314A9B00E8
:1017E0009B582F000436FEF784FFA4003D1B280001
:1017F000FEF7A8FD2A4B1B78002B01D0FEF74AFF0D
:101800003368019A1C121340264A9B009B582F00F4
:101810000436FEF76EFFA4003D1B2800FEF7CCFD4A
:101820001F4B28601B780435002B01D0FEF732FFD8
:101830003368019A1C1213401A4A9B009B582F00D0
:101840000436FEF756FF069B3D1DEB1A144CDB2BAE
:1018500004DD1A233D002370FEF71CFF02F022F97D
:1018600001234000184323783860002B01D0FEF795
:1018700011FF3368019A1C1213400A4A9B009B58BF
:101880002F000436FEF735FF069B3D1DEB1A044C76
:10189000DB2B09DD1A233D002370FEF7FBFEC0465B
:1018A00054020020F09E000002F0F2F8F64B4000D7
:1018B00018400123184323783860002B01D0FEF72D
:1018C000E9FE3368019A1C121340F04A9B009B58B2
:1018D0002F000436FEF70DFFA4003D1B2800FEF785
:1018E000B5FDEB4B28601B780435002B01D0FEF7CB
:1018F000D1FE3368019A1C121340E44A9B009B58A6
:101900002F000436FEF7F5FEA4003D1B2800FEF76D
:10191000B5FDDF4B1B78002B01D0FEF7BBFE336813
:10192000019A1C121340D94A9B009B582F00043681
:10193000FEF7DFFE0123A5007D1B20001A00290011
:10194000FEF7F0FDD34C2068643001F0EFFB002877
:1019500015D0029B21685A78CF4801F066FE15E049
:10196000A5007D1B2000012300222900FEF7DAFDDF
:10197000C84C2068643001F0D9FB002803D1043E34
:101980003D00FEF79AFEC44801F0EAFC0123029AEA
:10199000137002F07DF8C8222368D2000633534347
:1019A0001818029B5860FEF788FEFEF733FEB84B0E
:1019B000A4001B783D1B28600435002B01D0FEF7E6
:1019C00069FE3368019A1C121340B04A9B009B5871
:1019D0002F000436FEF78DFEA4003D1B280002F008
:1019E00095F8AB4B28601B780435002B01D0FEF72F
:1019F00051FE3368019A1C121340A44A9B009B5865
:101A00002F000436FEF775FEA4003D1B280002F0EF
:101A10007FF89F4B28601B780435002B01D0FEF720
:101A200039FE3368019A1C121340984A9B009B5858
:101A30002F000436FEF75DFEA4003D1B280002F0D7
:101A400069F8934B28601B780435002B01D0FEF712
:101A500021FE3368019A1C1213408C4A9B009B584C
:101A60002F000436FEF745FEA4003D1B280002F0BF
:101A70006FF8874B1B78002B01D0FEF70BFE336805
:101A8000019A1C121340814A9B009B582F00043678
:101A9000FEF72FFEA4003D1B280002F07BF87C4BD4
:101AA00028601B780435002B01D0FEF7F3FD336866
:101AB000019A1C121340754A9B009B582F00043654
:101AC000FEF717FEA4003D1B280002F095F8704BAE
:101AD0001B78002B01D0FEF7DDFD3368019A1C1244
:101AE00013406A4A9B009B582F000436FEF701FE04
:101AF0000121200002F068F8654B1B78002B02D012
:101B00003D00FEF7C7FD3368019A1C1213405F4A7F
:101B10009B009B580436FEF7ECFD0021200002F0EC
:101B200053F85B4B1B78002B02D03D00FEF7B2FD53
:101B30003368019A1C121340544A9B009B58043688
:101B4000FEF7D7FDA4003D1B280002F073F8504BB0
:101B500028601B780435002B01D0FEF79BFD33680D
:101B6000019A1C121340494A9B009B582F000436CF
:101B7000FEF7BFFDA4003D1B280002F06FF8444BA8
:101B800028601B780435002B01D0FEF783FD3368F5
:101B9000019A1C1213403D4A9B009B582F000436AB
:101BA000FEF7A7FDA4003D1B280002F031F8384BDA
:101BB0001B78002B01D0FEF76DFD3368019A1C12D3
:101BC0001340324A9B009B582F000436FEF791FDCC
:101BD000A4003D1B280002F071FD2D4B1B78002B4B
:101BE00001D0FEF757FD3368019A1C121340274AB3
:101BF0009B009B582F000436FEF77BFDA4003D1B85
:101C0000280002F0EFFD224B28601B780435002BE2
:101C100001D0FEF73FFD3368019A1C1213401B4AA6
:101C20009B009B582F000436FEF763FDA4003D1B6C
:101C3000280002F0F3FC164B1B78002B01D0FEF7B6
:101C400029FD3368019A1C121340104A9B009B58CF
:101C50002F000436FEF74DFDA4003D1B280002F0C6
:101C6000F3FC0B4B28601B780435002B01D0FEF7EA
:101C700011FD3368019A1C121340044A9B009B58C3
:101C80002F000436FEF735FDFEFFFF7FF09E0000BB
:101C9000540200205C02002060020020A4003D1BD2
:101CA000280002F0CBFAAA4B1B78002B01D0FEF7DC
:101CB000F1FC3368019A1C121340A64A9B009B5802
:101CC0002F000436FEF715FDA4003D1B280002F08E
:101CD000CBFA9F4B1B78002B01D0FEF7DBFC33685F
:101CE000019A1C1213409B4A9B009B582F000436FC
:101CF000FEF7FFFCA4003D1B280002F0C5FA944B40
:101D00001B78002B01D0FEF7C5FC3368019A1C122A
:101D10001340904A9B009B582F000436FEF7E9FCC5
:101D2000A4003D1B280002F0D7FA894B1B78002B3A
:101D300001D0FEF7AFFC3368019A1C121340854AAC
:101D40009B009B582F000436FEF7D3FCA300FD1A1E
:101D500029002000049302F0CFFD049B2860FD1AA7
:101D60007B4B04351B78002B01D0FEF793FC3368C6
:101D7000019A1C121340774A9B009B582F0004368F
:101D8000FEF7B7FCA300FD1A29002000049302F01F
:101D9000BBFD049B2860FD1A6D4B04351B78002B9E
:101DA00001D0FEF777FC3368019A1C121340694A90
:101DB0009B009B582F000436FEF79BFCA300FD1AE6
:101DC00029002000049302F0A7FD049B2860FD1A5F
:101DD0005F4B04351B78002B01D0FEF75BFC3368AA
:101DE000019A1C1213405B4A9B009B582F0004363B
:101DF000FEF77FFCA300FD1A29002000049302F0E7
:101E0000C5FB049B2860FD1A514B04351B78002B41
:101E100001D0FEF73FFC3368019A1C1213404D4A73
:101E20009B009B582F000436FEF763FCA4003D1B6B
:101E3000280002F079FA464B1B78002B01D0FEF700
:101E400029FC3368019A1C121340424A9B009B589C
:101E50002F000436FEF74DFCA5007D1B2900200055
:101E600002F014FB3A4B1B78002B01D0FEF712FC5A
:101E70003368019A1C121340364A9B009B582F006E
:101E80000436FEF736FCA4003D1B280002F0CAFA17
:101E90002F4B28601B780435002B01D0FEF7FAFB8E
:101EA0003368019A1C1213402A4A9B009B582F004A
:101EB0000436FEF71EFCA5007D1B2900200002F061
:101EC00093FA234B1B78002B01D0FEF7E3FB33681A
:101ED000019A1C1213401F4A9B009B582F00043686
:101EE000FEF707FCA5007D1B2900200001F0A0F8EB
:101EF000174B1B78002B01D0FEF7CCFB3368019AFF
:101F00001C121340134A9B009B582F000436FEF707
:101F1000F0FBA300FD1A29002000049301F088F8CB
:101F2000049B2860FD1A0A4B04351B78002B01D056
:101F3000FEF7B0FB3368019A1C121340054A9B0060
:101F40009B582F000436FEF7D4FB09B0F0BDC04605
:101F500054020020F09E00000023F7B55A1E0192A3
:101F6000002B07DA02F016F801F0D0FA01F082FB3C
:101F70006423019300263000194B19688E4201DB5F
:101F8000019BEBE7174B1A680132914200DC0022FB
:101F9000F0241A601D68144F6C43E35D002B1DD0C4
:101FA000E419022B16D0012B0ED1002801D101F02B
:101FB0006FFDF0226A430C4B0C499B185B68C31AF7
:101FC0008B4201D80223BB54F0235D43064BEB5CEC
:101FD000022B03D12000FEF735FBD1E70136CBE71A
:101FE0005802002000000020F81100209F86010008
:101FF000054B01211A68054B1A600023044AD15091
:102000000433642BFBD17047AC050020A4050020ED
:102010005023002000B59BB00200054901A807F03D
:10202000B7F801A801F0B8F901F024FBFCE7C046BD
:1020300030A1000037B5174D04002868002801D0F2
:1020400006F09AFCA400200006F08CFC2860002812
:1020500001D1114809E001AB984208D20F4B021997
:102060006B440193934202D20D48FFF7D3FF04283B
:1020700002D808302860083C2B680A4A1C191360F3
:10208000094B01211C600023084AD1500433642B02
:10209000FBD137BDAC05002041A100001CFCFFFFB7
:1020A00071A10000A4050020A805002050230020F5
:1020B00070B50D4D0D4E2B684C1CA40036681C19D4
:1020C000B44203D90A20FEF79FFA0BE02C601D00F2
:1020D000AC4201D904C5FBE70F22090110400843B7
:1020E0001860180070BDC046A4050020A805002097
:1020F0000322CB1C70B50C00D9171140C91805007C
:10210000891000220420FFF7D3FF0023A34204DA42
:10211000E95CC21811710133F8E7E1430023C917E4
:10212000214041180B7170BD10B5830706D10428FA
:1021300004D90F2304C81340042B03D00E20FEF74C
:1021400063FA014810BDC04681A2000070B50124A9
:102150000B680D001C4001D05C1002E00D20FEF762
:1021600053FA200005F058F8264904F041FF06F024
:102170001BFB02F02FFF0022234B05F0CFFC0023B6
:10218000002204F0FFFE01242B681C40002819D017
:10219000002C01D05C1002E00D20FEF735FA200083
:1021A00005F03AF8174904F023FF06F0FDFA02F0B3
:1021B00011FF0022144B05F0B1FC0022134B05F077
:1021C00073F818E0002C01D05C1002E00D20FEF73F
:1021D0001BFA200005F020F80A4904F009FF06F078
:1021E000E3FA02F0F7FE0022074B05F097FC00220D
:1021F000064B05F00DFF06F05FFA0123400018437F
:1022000070BDC046D30237390000D0400000E03F27
:1022100010B5034A0121034800F0F6FE10BDC04688
:1022200004000020DCA1000030B502248025094B09
:10223000094AED009C505C59002CFCD0A124E4001C
:10224000884204D28025ED0018514019F8E700219A
:10225000995030BD00E001400405000010B5002891
:1022600004D1E0209C210002890203E09C2080210F
:102270008002C902FFF7D8FF10BD002802D09C23BE
:102280009B0201E0E0231B021B6800201A0E532A68
:1022900001D11B02180A704730B501248025064A77
:1022A000064BED00D4505459002CFCD001600021A5
:1022B000014AD15030BDC04600E001400405000095
:1022C00010B5002802D09C20800201E0E02000022E
:1022D000A6230902DB05090A1943FFF7DDFF10BD3C
:1022E000F0B50124802503000F4F08000F49ED00D1
:1022F0007C507C59002CFCD09C46002810DD547882
:1023000016789378240234431B0423431C00D378AB
:1023100001381B062343644608C40432A446ECE794
:1023200000237B50F0BDC04600E0014004050000E2
:1023300070B505004B680A009C1C2100FFF7D0FF18
:10234000A000281870BD0000154B1B68002B04D09E
:1023500080219C23C9029B0203E09C21E023890287
:102360001B02002807D1191D5B6802001B0E522BAF
:1023700014D10A0012E0002281420FD903681B0E1B
:10238000522B0BD1436802339B00C318994205D9E5
:102390001A68110E0022522900D11A00100070474D
:1023A000B00700208022F0B5520085B000216248BD
:1023B00006F0F5FA802200215200604806F0EFFA9C
:1023C0005F4B1B681A00029353425A41100003925C
:1023D000FFF744FF029B002B01D15A4C00E05A4CFE
:1023E0000020FFF7B1FFFF270500002D00D194E08A
:1023F0002B681A121B143A403B4001921A000A3A09
:10240000092A43D84C4B019A995C002900D07FE0FF
:1024100010224E4806F0C3FA2E00336801991A12B2
:102420003A40914217D11A143A400B2A06D0132A87
:102430000CD00A2A0FD1454B1E600CE03B40022B0A
:1024400009DC424A9B00D3185E6004E010220021A0
:102450003E4806F0A4FA3000FFF776FF061EDCD1F6
:102460003A4B196800290FD02000FFF761FF0400E4
:10247000374E3168002903D02000FFF759FF0400D0
:10248000344B0436B342F4D12B4B3EE0143B092BC2
:102490003ED82A4B019A995C002939D108222E484E
:1024A00006F07DFA2E0033681A143A40152A0BD034
:1024B0001D2A11D0142A14D1019A1B123B409A42B2
:1024C0000FD1254B1E600CE0019A1B123B409A4233
:1024D00007D1214B5E6004E0082200211E4806F06F
:1024E0005EFA3000FFF730FF061EDCD11A4E31686D
:1024F000002909D02000FFF71BFF716804000029A4
:1025000002D0FFF715FF04000C4B0121019A9954EA
:102510002800FFF719FF050067E70298FFF7ADFEF7
:10252000411C0398FFF7CCFE054B039A1A600B4B36
:102530001C6005B0F0BDC046B0060020B00500200C
:10254000B00700200470020004E00000B423002063
:10255000B8230020C4230020C4230020B407002097
:1025600070B50020FFF789FE04000120FFF785FE0B
:10257000844200DA04000A4B1E6875427541280047
:102580001D60FFF76BFE002E01D0064B00E0064BEE
:10259000064A2800611C1360FFF792FE70BDC0461A
:1025A000B007002004E0000004700200B40700201F
:1025B000F8B50020FFF761FE07000120FFF75DFE80
:1025C0003E00224D0643224C0CD18021E020C9025E
:1025D0000002FFF729FE01213000FFF771FE2E6097
:1025E0001C4B2FE0874208DD00239C212B60194BF8
:1025F000890223602368002011E0012380212B60E1
:10260000154BC9022360F5E71A68551C18D0120E45
:10261000522A07D101205A68023292009B188B423D
:10262000F2D311E0002800D023600C4C0C492000AC
:1026300006F0DAFD200001F03DFAFFF791FF04E01B
:10264000002802D0236000E02160F8BDB007002020
:10265000B407002004E00000047002000024002001
:10266000F2A10000F0B585B0039203220333DC171A
:1026700014402A4EE3189C10336801900291002BFD
:1026800002D08022D20201E09C229202244FA51C9B
:102690003B68AD005B199A4217D2FFF783FE33689F
:1026A000002B02D08022D20201E09C2292023B68E1
:1026B0005B199A4209D21B4C1B49200006F094FD7D
:1026C000200001F0F7F9002026E0029B3E681B067F
:1026D000190C6B461A7BA423DB051343019A0B43A9
:1026E0001104FF221204114019433000FFF7D4FDFA
:1026F0003300301D0833210001933B60FFF7CCFD10
:10270000002C04D00A9A21000198FFF7E9FD30005F
:10271000019B083D5D193D6005B0F0BDB00700208C
:10272000B4070020002400201BA2000070B59AB05E
:10273000FFF73EFFFF221F4CD2000021200006F0D1
:102740002EF90020FFF700FEFF25002600281AD0F2
:1027500003681A142A400A2A08D11A122A40FF2AAA
:102760000ED0D200A1180B71A05009E0132A07D196
:102770001B122B40FF2B03D0DB00E2181671E65032
:10278000FFF7E2FDE2E7FF210200C900235808300D
:102790005D1EAB41D2188842F8D1074901A806F066
:1027A000F7FC01A800F0F8FD044800F0F5FD1AB0B0
:1027B00070BDC046581B002042A200005AA2000073
:1027C00000220121094B5A60094A51605A68002AC7
:1027D000FCD00022C021054B49001A61044B013294
:1027E0009A60044B01325A501A607047FC10004046
:1027F0000010004000E100E00222064B0121DA67F0
:102800000022054B5A61054A11615A69002AFCD021
:102810007047C04604E100E0FC100040001000409A
:1028200010B5054B1A781C00002A01D0FFF7E4FF11
:102830000023237010BDC04640080020024B1868DA
:1028400001234000184370473C08002000487047AF
:10285000E0230020024B1868012340001843704712
:102860007C00002070B504000D00160001F01AF97C
:102870008023012200215B055B6E6270E270020A18
:10288000A271020CE2711A0A60716372000EA272E8
:102890001A0C1B0E267025712072A170E272237330
:1028A00070BD0000124B10B51B68124C5A1C0FD0A3
:1028B000114C002B0CD0114C012B09D0104C022BC9
:1028C00006D00D4C042B03D00E4C052B00D10B4C25
:1028D00021000D4806F088FC200006F08DFC030066
:1028E000042204339B0809481B011343036010BDF5
:1028F0008000002024A300001DA300002FA30000DF
:1029000034A3000029A30000D0230020CC23002002
:1029100070B5214C2278002A3DD1204B01215A600C
:102920008022D20511605A68002AFCD000220720BC
:102930001B4B1C4901255A500439585008315A5034
:1029400019481A4958501A491A485A501A495A509F
:10295000A622D2009D50082218495A5004315850DE
:10296000022017495850174817495850174804393A
:102970005850182016495850C12189005A5005391D
:10298000FF395A58083802435A50124A124999508E
:10299000FFF716FF257070BD40080020FC000040C6
:1029A000001000400C050000746962751C050000F1
:1029B00024050000200004022C050000140500007E
:1029C00034050000FFFF00003C050000211001005D
:1029D0005405000004050000B807002010B50028C9
:1029E0000EDD0C68E3070BD56410FF2C08D8054BEF
:1029F0001B78002B01D1FFF78BFF034B034AD45008
:102A000010BDC04640080020240500000010004012
:102A100013B5002815DD0C68E30712D50822094913
:102A20006846641005F0B2FF072C0AD8064B1B78E5
:102A3000002B01D1FFF76CFF6B46044A1957044B7A
:102A4000D15016BD15A30000400800200010004022
:102A50000C05000010B5002813DD0C68E30710D545
:102A60006410532C0DD8074B1B78002B01D1FFF7B6
:102A70004FFFFFF7C1FEA123034ADB00D450FFF74D
:102A80009FFE10BD400800200010004070B50E4BA6
:102A900006001B78002B01D1FFF73AFF00200B4DF9
:102AA0002C7884420ED00A4B202219780323091B6C
:102AB0001940084B49015918300005F067FF012003
:102AC000013C2C7070BDC046400800204108002029
:102AD00038080020B8070020002330B589B098429C
:102AE00026DD03240D682C409C4221D12300042DB7
:102AF0001ED90F212A681140062919D112091F2A4F
:102B000016D96846FFF7C2FF2300002810D06B4695
:102B1000012019780123A14203DB6B461B5D5B009A
:102B20000343A200AA1801345360202CF2D10423DD
:102B3000180009B030BD0000F0B5424B8BB01B78D7
:102B4000002B01D1FFF7E4FE02AD2800FFF79EFF46
:102B5000002870D02B780B2B6DDD6B78012B6AD1A0
:102B6000EA780023012A66D1374F384C3B60237145
:102B70002B79374A1360002B0ED115256D446A78E6
:102B80002878AB78120202431B0413431A00EB7837
:102B90001B0613433B6050E0012B10D115266E44F9
:102BA00072783078B378120202431B0413431A0080
:102BB000F3781A261B0613433B606A7C25E0022B40
:102BC00002D16A7B162620E0042B0DD115210822A4
:102BD0006944684605F0DAFE0098019902F058F958
:102BE00005F06AFD386028E0052B26D11521082262
:102BF0006944684605F0CAFE0098019902F048F958
:102C000005F05AFD1E2638606A7D6E44132A00DDE9
:102C100013220023934204D0F05CE11808710133C1
:102C2000F8E704200021E21804339B101B01034342
:102C30001171236003E0002001E00022E9E70BB0FE
:102C4000F0BDC046400800203C080020E0230020E2
:102C50008000002010B5041E26D0144B1B78002BDA
:102C600001D1FFF755FEFFF7C7FD00201049114ABB
:102C7000114B8C5058600130086059680029FCD015
:102C800000200D4908610A4901308860196900294E
:102C9000FCD00A4B0A491B785B01CB1804498B50C6
:102CA000FFF7AAFDFFF78CFD10BDC04640080020CD
:102CB0000010004004050000FC100040380800200F
:102CC000B807002030B589B000281EDD03230A684C
:102CD00013401AD1042A18D90F2011680840062879
:102CE00013D109091F2910D9012401339900515822
:102CF0000020214201D04910C8B26D46591E6854C7
:102D0000202BF2D16846FFF7A5FF09B030BD30B5E2
:102D100089B0002826DD0868830723D1042821D93B
:102D20000F2302681340042B1CD1FFF7FDF90500A7
:102D300006F062FA041E122C00DD12242200022189
:102D40000D326846FFF78EFD6B465C730023A3428D
:102D500005DA1A00E95C6A4491730133F7E76846C3
:102D6000FFF778FF09B030BD70B50C0088B00128BE
:102D700033DD0868830730D104282ED90F23026879
:102D80001340042B29D14B68DB0726D5FFF7CCF97C
:102D9000060006F031FA6468050064100E2800DDB4
:102DA0000E252A00012111326846FFF75BFD6B46B4
:102DB0006A465C73231293732314D3730023240E87
:102DC00014745574AB4205DA1A00F15C6A449174CC
:102DD0000133F7E76846FFF73DFF08B070BD30B537
:102DE00089B0002814DD0C68E30711D510220021FA
:102DF0006846FFF737FD6B466A4665105D736846A7
:102E000063122D0E64149373D4731574FFF722FFAD
:102E100009B030BD184B10B55A681849002A03D0C4
:102E200000225A6001328A601B691448002B22D0AC
:102E30000023114A13618022D2008458104A012CC9
:102E400016D1A923DB00C3585B4213600D4A1378E7
:102E5000032B01D80133137003220B48037801338D
:102E600013400A4A03705B01D318094A8B5000E0F3
:102E7000136001238B6010BDFC1000400010004067
:102E80007C0000204108002038080020B8070020FE
:102E90000405000010B5034A0E21034800F0B4F801
:102EA00010BDC0460C0000203BA30000044A0549A9
:102EB0001368C85401339B059B0D13607047C046CF
:102EC000480C002042080020114A70B51368114CCC
:102ED000984211DA015D451CFA39012906D8AB4246
:102EE00006DD2118497801391F2901D92800EFE7AB
:102EF0000100251A461C02D10023136006E0665C1F
:102F00006E5401318B42FADC181A106070BDC04655
:102F10004C0C0020540C002010B500F0B9FD064BFD
:102F20001A68904201D200221A601B68C01A034B33
:102F300083428041404210BD500C0020204E0000D2
:102F400010B5094C094A2368126893420BD0084A0D
:102F5000D05C00F0D9FE002805D0236801339B0522
:102F60009B0D2360EDE710BD54100020480C00209D
:102F70004208002010B50400064B074A1B6812687F
:102F80009B1ADB439B059B0DA34202DAFFF7D8FF98
:102F9000F2E710BD480C002054100020F7B50600E1
:102FA0000191151E2FD05768B800441C0630FFF75A
:102FB000E1FFFB20FFF77AFF1C20FFF777FFF0B25D
:102FC000FFF774FFE0B22412FFF770FFE0B2FFF7E3
:102FD0006DFF6B461879FFF769FF0026BE4212DAD3
:102FE000B300EB189C680136E0B2FFF75FFF2012D8
:102FF000C0B2FFF75BFF2014C0B2FFF757FF200EEF
:10300000FFF754FFEAE7F7BD70B5074D2C68092CB0
:1030100008DC0C236343054E01349851F3185960C2
:103020009A602C6070BDC0465810002064240020B7
:10303000F0B589B004900E0001284BDD284B0868DC
:103040000293830709D1042807D90F23026813408C
:10305000042B02D1FFF768F80290214B70680393AC
:10306000830709D1042807D90F2302681340042BD2
:1030700002D1FFF759F8039000271A4B1A4D1B682D
:103080000593059B9F4225DA2B1F0299186806F0CD
:10309000A1F800281BD12B686C6806930190019B56
:1030A000069A934213DA20680399079406F092F87F
:1030B0000834002807D131000498079B08315B6869
:1030C0000238984709E0019B01330193E7E7013794
:1030D0000C35D6E71B20FDF797FA09B0F0BDC046C6
:1030E00081A20000581000206824002010B501F0D3
:1030F00041FA00F0C9FDFFF78BF800F033FEFFF74F
:10310000C9FE01F0AFFA01F065FC10BD962210B5C2
:1031100012010021034805F042FC0022024B1A6014
:1031200010BDC046F811002058020020064B074A87
:103130001B6812689B1ADB439B059B0D012283428F
:1031400000DC002210007047480C002054100020C2
:10315000F8B505000C0016001F1E0ED10320FFF766
:10316000E5FF002827D0FA20FFF7A0FEE8B2FFF71E
:103170009DFEE0B2FFF79AFE1DE0501DFFF7D6FF5F
:10318000002818D0FB20FFF791FEE8B2FFF78EFE73
:10319000E0B2FFF78BFEF0B2FFF788FE3012C0B24C
:1031A000FFF784FE3C00E31B9E4204DD2078FFF71E
:1031B0007DFE0134F7E7F8BD70B50024F0250B4B18
:1031C0001B689C420EDA2A006243094BD3181A7816
:1031D000002A05D05978002311201A00FFF7B8FF04
:1031E0000134ECE7FFF792FF70BDC04658020020A3
:1031F000F81100200123F3B50400FFB00D0010000A
:103200001A420DD002AA1370431002A95370421241
:103210001B0E40148A700B71C8700B00052273E0FE
:10322000032313401ED1042A1CD90F2201680A402F
:10323000042A17D1023302AA1370FEF775FF0600A5
:1032400005F0DAFFF823FF33984200DD1800002371
:10325000834205DA01335A1EB25C02A9CA54F7E769
:10326000421C50E0042801D0002809D1032302AAFF
:10327000043813704342434153701300022243E069
:10328000002B45D1042843D90F210268114005299C
:1032900012D1043302A90B70F8231209FF339200F4
:1032A0009A4200DD1A00002393422BDA0133C11841
:1032B000C97802AEF154F7E7062929D101390E0089
:1032C000120956430196F826019FFF36B7421FDCCC
:1032D00002AE31700136934213DA012701339900AF
:1032E0004158394201D0394100E00A49012737707D
:1032F0000F127170B7700F14090EF7703171053627
:10330000E9E7019A013202AB29002000FFF720FF14
:103310007FB0F3BD19FCFFFF70B5F023050000245A
:103320000D4A1800604380184178A94203D0013447
:103330000A2CF6D10FE0F022002105F030FB074AFD
:103340001368013BA34200D11460002329001A0036
:103350001120FFF7FDFE70BDF8110020580200207B
:1033600010B5B2B002236A460400137005F044FFA2
:10337000C72800DDC7200023834205DA69460133F0
:103380005A1EA25CCA54F7E7421C6B46FE21142069
:10339000FFF7DEFE32B010BD10B5B2B002236A46B0
:1033A0000400137005F028FFC72800DDC7200023A4
:1033B000834205DA694601335A1EA25CCA54F7E714
:1033C000421C6B46FF211420FFF7C2FE32B010BD35
:1033D000F7B5234B06001B68F0200093002321491A
:1033E000009A93420ADA02005A438A185478B44287
:1033F00002D11278002A31D10133F1E70024F02301
:103400001A00624301920199164A55182F78002F2D
:1034100006D001340A2CF3D11348FFF7BDFF1DE09D
:10342000F0223900280005F0BAFA02230D4A01996A
:10343000EB6053540D4AF1008A58009B6E70AE70D9
:10344000AA602F616F61A34202DC054B01341C604E
:10345000002331001A001020FFF77AFEF7BDC046A6
:1034600058020020F8110020F6A30000581B00208D
:1034700010B5FFF7A1FE0024064BE200D3181B791C
:10348000043B012B02D8E0B2FFF7A2FF0134FF2C6E
:10349000F2D110BD581B0020F7B50E0000247F2587
:1034A0000190194BE200D1180979062901D00329AE
:1034B00026D1985883682B401C2B21D1C3681A0051
:1034C0002A40042A1CD102692A40192A18D11B0A51
:1034D00001339B000C30C018FEF726FE070005F0F4
:1034E0008BFE0023B0420BD19E4206DD019AF95CAF
:1034F000D25C914204D10133F6E7E0B2FFF768FFF6
:103500000134FF2CCDD1F7BD581B002070B500F061
:10351000BFFA184B1A68904201D200221A601A684A
:103520001549821A8A4223D91860002000F082FBD4
:1035300044424441604207240443002000F08EFBD3
:10354000002810D0082600250C4BEA00D3181B7960
:103550009C4201D0B34202D1E8B2FFF739FF0135F6
:10356000FF2DF1D104E0631C02D001267642EAE788
:1035700070BDC046440C00200F270000581B0020DF
:1035800037B500240500FFF717FE01A8019400F0ED
:103590003FFB200000F068FE00F0FCFC00F072FB36
:1035A00000F071FB00F038FF00F09EFA0548FFF7CD
:1035B000F3FEA54204D0FEF71BFD0348FFF7ECFE27
:1035C00037BDC0460BA4000023A40000002310B5A3
:1035D00001001A001120FFF7BBFD10BD07B56B46B7
:1035E000197069465A7013128B701314120ECB7037
:1035F0000A716B46010005221320FFF7A9FD07BDE4
:1036000010B50A0001001220FFF7F4FD10BD70B5DF
:10361000050008000C003230FFF7ACFC2B00220044
:1036200000211B20FFF794FD70BD10B50C000300B6
:10363000110014202200FFF78BFD10BD70B50600AD
:103640000020FEF781FE0024FF25002810D003682B
:103650001A142A40152A05D11B122B40B34204D15B
:10366000040002E01D2A00D10024FEF76DFEECE705
:10367000200070BDF0B580279DB0FFF761FCB94D0B
:10368000B94C2868FF00391A201800F023FB2B687A
:103690000600C3182B60002B00D1DBE1002E0DDDEE
:1036A0002868391A201800F015FB2B6806001B1833
:1036B0002B6000F0EDF9AD4B1860EFE72378FA2BA3
:1036C00000D00CE12B68022B06DCFFF725FC00285C
:1036D00000D1BFE10120B8E16078A5780238182850
:1036E00000D9FAE003F08CFA0D1E22262932F93DAA
:1036F000676F7589DAEFF9F9F9F9F9F9F9F9F9F973
:10370000F300FF2D00D1E8E02800FFF705FE0022BE
:103710009749EB005A50CB181A71290000921300F8
:1037200013204DE02800FFF753FED6E02800FFF7F6
:10373000F3FDD2E0FFF79CFECFE0FFF73DFD002058
:10374000FFF71EFF8B48FFF727FEC6E0182D00D9B4
:10375000C3E0894BAA00D25829001520FFF74AFD83
:10376000BBE000242000FFF769FF071E03D10134EE
:10377000192CF7D1B1E0083005F03EFD0600053008
:10378000FFF7F8FBFB20FFF791FB1D20FFF78EFBF7
:10379000E0B2FFF78BFBF0B2FFF788FB3012C0B24C
:1037A000FFF784FB0025AE42E1DD7B19187AFFF7B5
:1037B0007DFB0135F7E700211D200B000A00009179
:1037C000FEF750FF89E00022290000921300272015
:1037D000F6E700F077F903AC684A64210090684B83
:1037E000200005F0A3FC02232000237005F004FD57
:1037F00023000200002116206DE000245C4AE30053
:10380000D558002D46D06B689E00701DFFF7B2FBA7
:103810002B0000253200083321000120FFF798FC1F
:103820000020FEF791FD2E002F0000281DD0FF2163
:1038300003681A120A40A24214D11A140A400B2A31
:1038400007D10B400DD0012B09D0022B00D1FFE096
:1038500008E0132A06D100252E002F0002E0060002
:1038600000E00700FEF770FDDFE7002E04D0320015
:1038700001212000FFF792FB002D04D02A00022135
:103880002000FFF78BFB002F04D03A00002120001E
:10389000FFF784FB0134FF2CB0D11EE0FFF78CFC56
:1038A0000025002429000094230022001320013564
:1038B000FEF7D8FEFF2DF4D1FF222100D2002C48C4
:1038C00005F06DF809E00120FFF75AFE05E000233E
:1038D00029001A001A20FFF73BFC0320B5E0FB2B60
:1038E00000D0F7E62A68042A00DCEEE62679E078C4
:1038F000244B360206439E4200DDEBE6331D9A421E
:1039000000DCE2E6E35CFE2B00D0E3E66078A5781D
:10391000731E1C2868D007D8082835D01B285ED015
:10392000012800D090E007E01E2800D17EE066D399
:103930001F2800D180E087E0FF2D00D184E028001F
:10394000FFF7EAFC67790634B31E290000943A00B9
:103950000A20FEF787FE064BED00E8505D192F7137
:1039600072E0C0464C0C0020540C0020500C00208B
:10397000581B002033A40000502300204AA400005C
:1039800045A40000F6030000182D5DD860790228D8
:1039900013D003281BD0012856D1A71D7A78A4790B
:1039A000BB78120222431B0413431A00FB78AD00BC
:1039B0001B0613435B0003430EE0002B44DDB11EE6
:1039C000A01DFEF795FB244BAD00E8503CE0A37929
:1039D000AD005A1E93419B001F4AAB5034E0601D5E
:1039E0001900FFF759FD2FE0FF2D2DD06279022A33
:1039F0002AD80634B31E009429000B2022E0632B42
:103A000000DD6323002203A8934204DDA118497955
:103A100081540132F7E7D9430022C91719404118F0
:103A20000A7001330090290015200BE00534009442
:103A3000002229001E2005E0042B05D100222900C8
:103A400005340094FEF70EFE701DFFF73DFA01E00D
:103A5000050007E71DB0F0BD50230020002070478F
:103A6000002070470020704700207047012200208E
:103A7000054B06491A6158500330043158508018DC
:103A8000083158501A60704700800040040500005B
:103A90000122034B1A64A822D20098587047C046EE
:103AA0000080004010B5FFF7F3FFFA21890003F012
:103AB000B1F810BD10B50100014802F055FE10BD6F
:103AC00084110020004870475CA4000070B5054ECA
:103AD0000400335C0D008B4202D002F06DFD3555C1
:103AE00070BDC0465C10002070B50024064D635DBB
:103AF000012B05D10021200002F05EFD002363555B
:103B000001341D2CF2D170BD5C1000200D207047D7
:103B10003B207047036870B55B100120052B12D85D
:103B2000094A9B009C58094D2B5D002B05D00021B4
:103B3000200002F041FD00232B55200002F0E6FB9F
:103B400001234000184370BD8CA400005C100020CD
:103B500070B5036845685C106D1004D40B4B9D4232
:103B600002DD1D0000E000251C2C0DD8084E335D41
:103B7000012B05D00121200002F01EFD0123335549
:103B80002900200002F050FC70BDC046FF03000079
:103B90005C10002070B5046864101C2C0FD8094D0F
:103BA0002B5D002B05D00021200002F005FD002335
:103BB0002B55200002F034FD0423012800D00023FF
:103BC000180070BD5C10002070B504000D001C28AA
:103BD0000ED8084E335C012B04D0012102F0ECFC1E
:103BE00001233355290020004D1EA94102F002FD9A
:103BF00070BDC0465C100020436810B5191F4A42D2
:103C00004A41006811004010FFF7DEFF10BD0000C0
:103C100037B569460200064B684630CB30C11368A1
:103C2000042B02D100F030FB01E000F055FB37BD62
:103C300054A4000010B5084C6379002B05D0002176
:103C4000052002F0B9FC00236371052002F0E8FCB6
:103C500043425841800010BD5C10002010B5084C54
:103C6000E37A002B05D000210B2002F0A5FC0023F5
:103C7000E3720B2002F0D4FC43425841800010BD97
:103C80005C1000207047704710B5034A04210348B8
:103C9000FFF7BAF910BDC046840000204BA3000016
:103CA000E12110B54902094802F0A5FDFFF7DEFE4B
:103CB0000A2002F025FB0023FF21054A9954013315
:103CC0001D2BFBD100F0A8FB10BDC04684110020C5
:103CD0005C100020F8B50B4E070030000D0002F01C
:103CE000C9FD041EAC4200DD2C003D00EB1B9C42D4
:103CF00005DD300002F0C8FD28700135F6E7200030
:103D0000F8BDC0468411002010B50100014802F042
:103D100079FD10BD841100200020704710B51E20D1
:103D2000FCF772FC10BD10B51E20FCF76DFC10BD39
:103D300010B51E20FCF768FC002010BD10B51E2039
:103D4000FCF762FC10BD10B51E20FCF75DFC10BD39
:103D500010B51E20FCF758FC10BD10B51E20FCF756
:103D600053FC10BD10B5034A08210348FFF74CF976
:103D700010BDC046A4000020A4A400000123034AF3
:103D80001360034A1068984018437047841000205D
:103D90008C100020202800D90020084B8000C25839
:103DA00001239340064A07491360074A1160074AF6
:103DB00007491160074A13607047C0467CA900009C
:103DC00080100020080500509C1000209410002056
:103DD0000C05005018050050F0B5EFF310810123D9
:103DE000194083F31088134E134AB4461268013AFF
:103DF0009340124A1468124A1568124A002B15D0D3
:103E0000166803420BD02660C046C046C046C04676
:103E1000C046C046C046C04616682E6004E06746ED
:103E20003E601668084F3E605B08E7E781F3108844
:103E3000F0BDC04608050050EC0000209C1000209A
:103E400094100020801000200C05005030B585B083
:103E500001AD0C220649280004F098FD0024285DDD
:103E600001210134FFF732FE0C2CF8D105B030BD32
:103E70001AA50000F0B53B4C85B0210003220C319F
:103E8000684604F083FD210009220F3101A804F0E7
:103E90007DFDFFF707FE344B344CC0182368984271
:103EA00001D2002323602568002D3ED12E006B46F1
:103EB00004339F5D01213800FFF708FE0136012120
:103EC000380002F097FB092EF1D100266B469F5D6A
:103ED00001213800FFF7FAFD01360021380002F019
:103EE00089FB032EF2D1C82080000138C046C046AD
:103EF000C046C046C046C046C046C046C046C04692
:103F0000C046C046F1D100210420FFF7DFFD0026A6
:103F10006B460021985D0136FFF7D8FD032EF7D1DF
:103F2000FFF7C0FD1330206019E0FFF7BBFD2368E9
:103F30000025984213D3042002F0E8F90C4B0D4EF3
:103F4000C01801D4306000E035603068032102F011
:103F5000EBFE00230125084A30602360136028002F
:103F600005B0F0BD1AA50000102700007C1000204D
:103F7000C8FEFFFF8C1000208410002010B5012423
:103F8000044001D0441002E00D20FCF73DFB20006E
:103F900010BD00007FB5A44E3368002B0BD1A34A9F
:103FA0001268002A07D1A24B1B68002B00D139E10F
:103FB000FFF760FF36E19F4D2A68002A2AD19C4A0C
:103FC0001268002A07D0FFF755FF002800D129E129
:103FD000FFF73CFF05E0954A1268002A01D1002B4B
:103FE000F6D1924B19681A00002911D03468002CC0
:103FF0000ED101AD0C22904928001C6004F0C6FCD3
:10400000285D00210134FFF761FD0C2CF8D109E196
:104010003368136000211A2002F0ECFA00211B2003
:1040200002F0E8FA00211C2002F0E4FA2E68012ECA
:1040300056D0022E00D19CE0002E00D0ECE00136DC
:1040400031007A4C03202368994302F0D3FA04200C
:10405000216801400B005942594102F0CBFA10216E
:1040600023680A200B405942594102F0C3FA8021CB
:10407000236809010B4059425941062002F0BAFA5F
:104080008021236809020B4059425941072002F060
:10409000B1FA8021236849020B4059425941092055
:1040A00002F0A8FA8021236889020B405942594145
:1040B000192002F09FFA80212368C9020B4059425F
:1040C0005941182002F096FA802321681B030B4007
:1040D00059425941172002F08DFA31001A2099E017
:1040E0000221524C172023680B405942594102F0DB
:1040F00081FA0821236818200B405942594102F0E7
:1041000079FA80212368C9000B40594259410420A3
:1041100002F070FA8021236849010B40594259414D
:104120000A2002F067FA80212368C9010B40594236
:104130005941032002F05EFA8021236889030B4075
:1041400059425941092002F055FA802321681B0485
:104150000B4059425941192002F04CFA3100062017
:1041600002F048FA3100072002F044FA31001B2027
:1041700050E020212D4C172023680B405942594113
:1041800002F038FA4021236818200B405942594167
:1041900002F030FA8021236819200B40594259411E
:1041A00002F028FA8021236849000B405942594106
:1041B000092002F01FFA8021236889000B40594230
:1041C0005941072002F016FA8021236889010B402B
:1041D00059425941062002F00DFA80212368490313
:1041E0000B40594259410A2002F004FA8021236809
:1041F000C9030B4059425941032002F0FBF98023C7
:1042000021685B040B4059425941042002F0F2F945
:1042100001211C2002F0EEF92B680321581C02F04A
:1042200069FE29607FBDC0469010002088100020E4
:1042300084100020981000201AA50000006810B516
:10424000C30703D5FFF79AFE054B1860054B1B68A3
:10425000002B03D0024B186800F0BAFB10BDC0461B
:1042600090100020A41000200022054B10B51A6009
:10427000044B1B68934201D000F0A8FB10BDC04660
:1042800090100020A410002070B505000068FFF712
:1042900075FE04006868FFF771FE631E0100042BC1
:1042A00014D8451E042D11D805226A43D3180122C3
:1042B00015009D402B00064805682B430360054B05
:1042C0001B68002B02D0200000F081FB70BDC046AF
:1042D00090100020A410002070B505000068FFF7C2
:1042E0004DFE04006868FFF749FE631E0100042BC1
:1042F00014D8451E042D11D805226A43D318012273
:104300009A401300064802689A43064B02601B68F5
:10431000002B03D00022200000F059FB70BDC046E6
:1043200090100020A41000202C4BF7B51B6804004F
:10433000002B03D101204042FFF72CFD0126246809
:10434000344219D0FF226310180212041040FF22D9
:10435000611212020A40DBB210431843204B1B6863
:10436000202B06D1B4401F4BA40EA400E35800023A
:104370001843FFF731FD30E0032525402DD1042CF3
:104380002BD90F2322681340062B26D1FF271309B0
:1043900001933F04019B9D421FDAAB00E3185A686A
:1043A000324218D0531018023840FF2184460902C7
:1043B000501208406146DBB208431843084B1B68A3
:1043C000202B06D15200920E064B9200D3580002C9
:1043D0001843FFF701FD0135DCE7F7BD8010002031
:1043E000EC00002048A500000B6810B50200D807BB
:1043F00001D5581001E0012040421823012A03DDB5
:104400004A68042A00D10833024A1360FFF7C2FC4D
:1044100010BDC046EC000020012010B54042FFF75F
:10442000B9FC10BD0068F8B5C30702D5FFF7A6FDBB
:104430000BE0830726D1042824D90F2203681A40F1
:10444000042A1FD11B091DD000790300203B5E2BDD
:1044500018D80522002053430B4E9D18043AAB4256
:104460000CD0052110249F5D3C4200D080180139FA
:10447000520064100029F7D10133F0E70123400016
:10448000184300E00120F8BD48A60000F0B5050083
:1044900085B008680C00FFF771FD0390022D08DD60
:1044A0006068FFF76BFD0700A068FFF767FD040079
:1044B00001E00124270005236343053B0293012308
:1044C00026000193231D9E4234DC3D003B1D9D428E
:1044D0002BDC731E042B23D86B1E042B20D8029BCD
:1044E000039A591E019B49191A40204B0AD00122F8
:1044F0008A4019680A431A601D4B01221B68002B71
:104500000ED009E001208840010018688843186037
:10451000174B1B68002B03D03100280000F057FA1E
:10452000019B01355B000193D0E7029B0136053307
:104530000293C7E73D1D042D15D8012C13D1260089
:104540003300AB40094A11689943094B11601B685D
:10455000002B04D0781D0022210000F038FA01342D
:104560000535062CECD105B0F0BDC04690100020FA
:10457000A410002010B5034A01210348FEF744FDB2
:1045800010BDC046E400002032A500000122094B06
:104590001A60094A1368002BFCD00322074B1B68E2
:1045A000D8171040C0180123801006384000184367
:1045B0007047C04600C0004000C1004008C5004030
:1045C0000120704710B5064C200000F039FB05496A
:1045D000200000F059FB0122034B1A6010BDC046B9
:1045E000C8100020801A0600A010002010B501217C
:1045F0000D20FFF76BFA01210E20FFF767FA00216B
:104600000F20FFF763FA044C200000F055FA102148
:10461000200000F06DFA10BDB410002010B5046841
:104620000D20E30703D56410FF2C03D91720FBF7F7
:10463000EBFF06E0FFF7DAFFE1B2024800F07AFA9A
:10464000002010BDB410002010B5FFF7CFFF0021EF
:10465000034800F06FFA01234000184310BDC04624
:10466000B410002010B5034A07210348FEF7CCFC24
:1046700010BDC046F400002023A800000D4B70B50B
:104680001B6804000E001500002B01D1FFF79AFFF4
:10469000E1B2094C200000F07FFBF1B2200000F0F5
:1046A00090FAE9B2200000F08CFA200000F0DEFB66
:1046B00070BDC046A0100020C810002010B5012415
:1046C0000368234205D04168214202D08268224219
:1046D00001D10D2004E058104910802803D915207D
:1046E000FBF792FF0BE0FF2901D91620F8E75210E3
:1046F000FF2A01D91720F3E7FFF7C0FF002010BD04
:10470000F7B501242300A04237DD0A68144234D0F3
:104710001B4B55101B684C68002B01D1FFF752FF53
:104720000127184EE9B2300000F036FB3C4205D0BC
:104730003C413000E1B200F044FA1AE00325254084
:1047400017D1042C15D90F2322681340062B10D142
:1047500013090193019B9D420BDAAB00E3185968E2
:10476000394204D04910C9B2300000F02AFA0135AC
:10477000F0E7300000F07AFB00231800FEBDC046D1
:10478000A0100020C8100020144B70B51B68050055
:104790000E00002B01D1FFF715FF114CEDB22900DF
:1047A000200000F0F9FAF1B2200000F00AFA00212E
:1047B000200000F0FDFA002801D040420CE0012268
:1047C0002900200000F0E3FA200000F0F0F90028B2
:1047D000FAD0200000F0F0F970BDC046A010002013
:1047E000C810002010B501240368234202D041689C
:1047F000214201D10D2004E058104910802803D92E
:104800001520FBF701FF07E0FF2901D91620F8E783
:10481000FFF7BAFF4000204310BD0000002370B531
:10482000344D0400EB5601332BD10D211D20FFF731
:10483000ABFF5A2804D101222A212A703D380AE010
:104840000F211920FFF7A0FF332807D102235F2291
:1048500020212B701A38FFF711FF12E00D211E20C6
:10486000FFF792FFC7280AD1032300222A21A93883
:104870002B70FFF703FF1B222A211E20EBE70023EA
:104880002B700023EB56022B06D0032B13D0012BE9
:1048900026D121001D2010E0012C04D1292119204E
:1048A000FFF772FF0DE0032C15D12B211920FFF724
:1048B0006BFF043C05E021001E200124FFF764FF8C
:1048C00064427F2801DD0138FF3803007F330ADAB4
:1048D0007F20404207E0052C02D12D211920ECE772
:1048E00001240020644264237F21584302F01CFA13
:1048F000604370BDF000002010B50120FFF78EFF6F
:1049000001234000184310BD10B50320FFF786FFB8
:1049100001234000184310BD10B50520FFF77EFFAE
:1049200001234000184310BDF8B501263400B04201
:1049300036DD0F683E4233D04D68AB0730D1042DD1
:104940002ED90F232A681340062B29D1154B1B683B
:10495000002B01D1FFF736FE0024354204D12B682D
:104960001C09202C00D920240F4E7F10F9B2220000
:10497000300000F00CFAA700EF19AF420DD0300064
:1049800000F015F90028FAD0300000F015F90123E5
:104990004000184368600435EFE7012064000443D9
:1049A0002000F8BDA0100020C81000200020704793
:1049B000002070470020704700207047002070479B
:1049C00000207047002070470020704770477047F4
:1049D0007047000010B5034A08210348FEF714FB96
:1049E00010BDC0462C01002064A8000010B5FFF7E0
:1049F00057F9AF20C000FDF71DFBFEF777FB044819
:104A0000FEF7CAFCFDF792FEFEF732FD10BDC04670
:104A10000BA4000010B5FDF79FFA10BD70B500257E
:104A200004AC24780573A94205D10A4B0A4A232114
:104A30000A4803F02BFF01600949920052589B007D
:104A400002715B588371A3005B5885604371022338
:104A5000C37170BDE7A80000AAA80000F5A8000077
:104A60007CA90000037B002B04D143738373036193
:104A700001330373704700001FB50191A02100248A
:104A80000068C900D2B24450012A07D0A24203D024
:104A9000032A05D1042202E0022200E00622134389
:104AA000034A8350034B019AC250012343501FBD58
:104AB000540500002405000010B50400FFF7D2FFE4
:104AC000A1222368A179D20099506179064A200079
:104AD0009950217904329950044B19685A689B689F
:104AE000FFF7CAFF10BDC0460C050000A81000204B
:104AF0004BB2002B0CDB80233F290CD81F290CD88C
:104B00000F290CD807290CD803290CD81B060BE059
:104B100080239B0408E0DB0406E01B0504E05B0542
:104B200002E09B0500E0DB050168014A8B507047FD
:104B3000240500000368074A99501A00FC32D16826
:104B40000029FCD0A321C90058580023C0B2D3606B
:104B50007047C0461C05000007B58022074BD205F0
:104B60001A6000229A6002321A710F230C320093ED
:104B70000349023B0348FFF751FF07BDA81000207F
:104B800000300040B4100020F8B505000E001700FA
:104B90000024BC4208D02B68315D1B682800984770
:104BA000002801D00134F4E72000F8BD704710B5AB
:104BB0001C3001F005FE10BD10B51C3001F0F2FDF7
:104BC00010BD70B5437E0D00002B05D0643004008D
:104BD00001F005FE002801D0002004E0200029009B
:104BE00001F0D1FD012070BD10B51C3001F0EEFDCB
:104BF00010BD0000F7B50193FA23002504009B00C7
:104C000083600D4B4560083303601C300F001600B5
:104C100001F0AEFD2000643001F0AAFD074AB600A5
:104C2000B35827616375019B20009B009B586576F4
:104C3000A576A375FEBDC0465CA900007CA9000056
:104C40000123A022C375837D0C49C133FF33D205F4
:104C50009B009950437DC133FF339B009950CC2179
:104C60000369074A490499500521243A9950817DE6
:104C700008329950417D034A995070470C06000054
:104C8000240500000C050000A02302690020DB00C1
:104C9000D0500948814204D90848814204D9CD2125
:104CA00003E0CC21490401E08021C90404481150EB
:104CB0000521D1507047C046A086010090D0030066
:104CC00024050000F7B5050000200C000193824286
:104CD0005CD0161E402E00D940262F001C3738000D
:104CE00001F05CFDB1222B69D20080219C50012291
:104CF00089005A50A97E002901D11A621A60002445
:104D0000731E2A69A34206D1019B002B03D0802386
:104D100002219B00D150012313621300FC33D96898
:104D2000002902D1996A0029F9D0996A00290AD18B
:104D3000D960A323DB00D1583800C9B2013401F097
:104D400022FDA642DCD8019A2B69002A04D11A0060
:104D5000FC32916A00290AD001210022AA76596109
:104D60001900FC3188680028FCD08A6007E0012126
:104D7000A976D961D16C0029FCD00021D164FC3323
:104D80009A6A002A01D000229A62E0B2FEBD10B5F4
:104D90000123FFF797FF10BD0300AC3310B50400EB
:104DA0001970643001F0FAFC0123637610BD000035
:104DB000F8B500220D0001004276AC310369040011
:104DC0000878B121C9005850802189005A50013219
:104DD0001A629A6026006436300001F0F1FC002867
:104DE0000ED03000276901F0DDFC1E4BF85023691E
:104DF000FC331A6A002A0CD19A6A002AF9D008E01A
:104E00002369002D0AD11A00FC32916A002905D1CC
:104E10000EE09A6A002AF3D11A62DBE701225A6196
:104E20001A00FC3291680029FCD00021916006E054
:104E30000121D961D16C0029FCD00021D1641A0074
:104E40000020FC32916A81420BD0074990625A5887
:104E500002305A50824204D0043A53425341023045
:104E6000C01AF8BD1C050000C404000010B50121E3
:104E7000FFF79EFF10BD000010B513231422024956
:104E80000248FFF7B7FE10BD00400040C8100020E8
:104E9000F0B5474680B4CB0F98464A4C4B005B0DAB
:104EA0001E1982B007000A00132E35DC002E57DBD6
:104EB000454B040033411F000F4007430D00002FF6
:104EC00024D05B081C000C4020430027002807D09A
:104ED000132E00D172E08022D202324199430A435C
:104EE0004346DE00394B11009E193468756838005E
:104EF00022002B0002F0D8F900900191009801994E
:104F000022002B0003F084F804000D00200029008B
:104F100002B004BC9046F0BD332E0CDD80230400AB
:104F20000D00DB009E42F1D102000B0002F0BCF943
:104F300004000D00EAE7264C0D00A446012463445A
:104F40006442DC40A446614604000142DED04908C8
:104F50000142C5D08027FF051F4188430743BFE7B3
:104F60004B005B08034304000D00002BCED00B0365
:104F70001B0B03435A42134380221B0B12031340A3
:104F80004A0C5204134319004346104ADB00D3185D
:104F90001C685D6822002B0002F086F900900191E8
:104FA0000098019922002B0003F032F842464B0092
:104FB0005B08D607334304001D00A7E780273F06A0
:104FC00089E7C04601FCFFFFFFFF0F0000AA0000B9
:104FD000EDFBFFFF30B5214A4B0087B05B089342E1
:104FE0001EDD1F4A934205DD02000B0003F010F89E
:104FF00007B030BD02AA00F035F803231840049A28
:10500000059B01281ED0022811D000281FD002982D
:10501000039900F02DFA80231B069C466144E7E7C4
:10502000002300220093002300F088FFE0E7012422
:1050300002980399009400F081FF80231B069C4690
:105040006144D5E70298039900F012FAD0E70124F1
:1050500002980399009400F071FFC9E7FB21E93F32
:10506000FFFFEF7FF0B54E4657464546E0B4DC4BB8
:105070004E0090B01700894676089E4200DC81E021
:10508000D84B9E4220DCD84A002900DC89E1D74B6E
:1050900002F0BEFFD54B04000D009E4200D18AE015
:1050A000D34AD44B02F0B4FF02000B0020003A6058
:1050B0007B60290002F0ACFFCD4ACE4B02F0A8FF86
:1050C000B860F960012066E0CB4B9E4200DC8DE0C9
:1050D000CA4B9E4265DCCA4932158A469244534601
:1050E0001B05F51A2900040003F0E6FA03F01AFB89
:1050F00002000B00200029000A920B9302F088FFA7
:105100000022C04B02F00AFD0290039103F0D4FA92
:1051100003F008FB04000D0002000B000298039945
:105120000C940D9502F074FF0022B64B02F0F6FCD1
:10513000002200230E900F9101F000FF002800D103
:105140004CE1002300222000290001F0F7FE02229A
:10515000431E9841131AAC4A3900019202220AA850
:105160000092524600F09EFA4B46002B13DA802242
:10517000120694467B68404263447B60FB6863444C
:10518000FB6008E002000B003A607B600022002315
:105190000020BA60FB6010B01CBC90469946A24645
:1051A000F0BD02000B0002F033FFB860F960386018
:1051B00079600020EFE7D3228E4B520502F028FFE2
:1051C000924A934B04000D0002F022FF02000B00F4
:1051D00020003A607B60290002F01AFF8B4A8C4B5A
:1051E00002F016FFB860F9600120D4E700F056FF26
:1051F000884A894B04000D0002F090FC0022874B86
:1052000002F052F803F058FA804603F08BFA764A1F
:10521000764B0690079102F081FC02000B00200003
:10522000290002F0F5FE734B02900391069807994E
:105230006F4A02F073FC434604000D000494059588
:105240001F2B30DC013B764A9B009B589E422AD0A4
:1052500002000B000298039902F0DAFE02000B0034
:1052600005000C003A607B60029803992A00230035
:1052700002F0CEFE049A059B02F0CAFE06000B0067
:105280003200BA60FB604B464046002B00DB82E7F1
:1052900080231B069C46644461443D607C60BE6084
:1052A000F960404277E7049A059B0298039902F05F
:1052B000AFFE0B0002003A607B604B0036155B0DC1
:1052C00005000C00F31A102BCEDD06980799D322A7
:1052D000484B520502F022FC04000D0002000B00B6
:1052E0000298039902F094FE02000B0002980399C1
:1052F0000892099302F08CFE22002B0002F088FE37
:1053000004000D0006980799404A414B02F006FC44
:1053100022002B0002F07CFE02000B00049005919D
:105320000898099902F074FE02000B003A607B6055
:105330004B005B0DF61A0500089A099B0C000292BF
:105340000393312E90DD06980799B822304B9205D1
:1053500002F0E4FB04000D0002000B000298039928
:1053600002F056FE0A0001001300029103920200AF
:105370000898099902F04CFE22002B0002F048FE2A
:1053800004000D0006980799264A274B02F0C6FB39
:1053900022002B0002F03CFE02000B000492059359
:1053A00058E7124B01F080FF104B04000D009E42A5
:1053B0003CD00F4A0F4B01F077FF02000B0020009A
:1053C0003A607B60290002F023FE094A094B01F094
:1053D0006BFFB860F96001204042DCE60323BAE6C7
:1053E000FB21E93F7BD9024000004054FB21F93FFB
:1053F0003163621A61B4D03DFB213941FFFFEF7F79
:10540000EAFBFFFF0000704190AA00007370032EBA
:105410008A19A33B83C8C96D305FE43F0000E03FB9
:1054200010AA0000C14920259A837B39D3220D4B55
:10543000520501F039FF0C4A0C4B04000D0001F03D
:1054400033FF02000B0020003A607B60290002F06D
:10545000DFFD054A054B01F027FFB860F960012028
:10546000404298E661B4D03D7370032E8A19A33B85
:10547000F0B54F464646C0B487B000920193754BD5
:105480004F00814688467F089F4263DC03F014F991
:10549000002800D1DAE04A4643464846414602F039
:1054A0003DFB04000D006C4A6C4B02F037FB6C4A6C
:1054B0006C4B01F0F9FE22002B0002F02FFB6A4A30
:1054C0006A4B02F0A5FD22002B0002F027FB684A80
:1054D000684B01F0E9FE22002B0002F01FFB664A38
:1054E000664B02F095FD22002B0002F017FB644A88
:1054F000644B01F0D9FE22002B0002F00FFB02905A
:1055000003910022604B2000290002F007FB029A61
:10551000039B06000F002000290002F0FFFA009A0A
:10552000019B04000D004846414602F0F7FA0200D4
:105530000B002000290002F06BFD02000B00300080
:10554000390002F065FD02000B0000204F4902F017
:105550005FFD70E002000B0002F0E0FA04000D00B5
:105560003D4A3E4B02F0DAFA3D4A3E4B01F09CFECA
:1055700022002B0002F0D2FA3B4A3C4B02F048FDDD
:1055800022002B0002F0CAFA394A3A4B01F08CFE95
:1055900022002B0002F0C2FA374A384B02F038FDE5
:1055A00022002B0002F0BAFA354A364B01F07CFE9D
:1055B0002B00220002F0B2FA354B029003919F4279
:1055C0009FDD344B00229F423ADC334900207B1898
:1055D0002E4916001F0002F01BFD049005910022C9
:1055E000294B2000290002F099FA32003B0002F01A
:1055F0000FFD029A039B06000F002000290002F015
:105600008DFA009A019B04000D004846414602F0C5
:1056100085FA02000B002000290002F0F9FC0200CC
:105620000B003000390002F0F3FC02000B0004987C
:10563000059902F0EDFC07B00CBC90469946F0BD10
:10564000164B002604920593154FC8E700200F491A
:10565000F1E7C046FFFF3F3ED43888BEE9FAA8BD57
:10566000C4B1B4BD9EEE213EAD529C804F7E923EB1
:105670009015CB19A001FA3E7751C1166CC1563F67
:105680004C5555555555A53F0000E03F0000F03FF3
:105690003233D33F0000E93F0000E0FF0000E73F66
:1056A0000000D23FF0B556464D4644465F46F0B442
:1056B0008E4CA544099119001400A89A0B938C4BA9
:1056C0009200D2580B000290013BE01E18211D00F1
:1056D00016000892009301F027FBC3430200DB177A
:1056E0001A401300110001330E929A009B1ADB003E
:1056F0001B1906934C1B761918D4A99BA5009C4630
:10570000361926AF6544013607E0286803F00AF829
:10571000013403C70435B44208D0002CF5DA002068
:105720000021013403C70435B442F6D1089B002B95
:1057300001DA00F0F9FB76AB19008B4626AA9146F8
:10574000089A0A930132D2009344029A9A469046EC
:10575000009BDB00994408339844009B002B00DA3F
:10576000B5E14C4600260027029D2268636803CD00
:1057700002F0D4F902000B003000390001F094FD72
:10578000083C06000F004545EFD15346C0C39A467A
:1057900008239C46E144DA45DFD10899554A0B00BD
:1057A000944663449B0012A884461A0002986244FF
:1057B00083460D920B9A0433D200634493440F93B3
:1057C0000591059A0A98D30019000C938C460300A2
:1057D00063441E685F68002A34DD12AB99461300EB
:1057E000454A804694466344DB00984474AB9A462D
:1057F0000022424B3000390002F090F902F05CFFC9
:1058000002F090FF00223E4B04000D0002F086F9EA
:1058100002000B003000390002F0FAFB02F04CFFEE
:105820004B4601C39946434620001A685B6829002D
:1058300001F03AFD08235B429C46E04406000F005D
:10584000D045D5D1069B30001A003900994600F0AA
:10585000C1FCFF2300229B0504000D0002F05EF94D
:1058600000F020FC0022274B02F058F902000B0048
:105870002000290002F0CCFB04000D0002F01CFF08
:10588000804602F04FFF02000B002000290002F0CA
:10589000BFFB4C4606000F00002C00DCF8E0059B27
:1058A00018205A1E920012AB9B58001B1900014190
:1058B000884481405B1A12A98B501722121B134196
:1058C0000793079B002B4BDD01239C46059BE0447F
:1058D000002B00DCF2E280251096119712AB00211C
:1058E000002409486D04059F19E0C04684FDFFFFB0
:1058F00098AB0000FEFFFF3FFFFFFF1F0000703E60
:105900000000704100002040FFFFFF00002A02D08D
:10591000AA1A1A600134013104338F4209DD1A6872
:10592000002CF3D0821A01311A60012404338F4213
:10593000F5DC109E119F069B002B0EDD012B00D184
:10594000B1E0022B09D1059B12A95A1E920012AB9D
:105950009B5810939B029B0A8B50079B022B7ED077
:10596000002300223000390001F0E8FA059B0028EE
:1059700000D16BE208995A1E914210DCBF490F9882
:105980008C4612A963448C4600219B0063441C682A
:10599000043B21438342FAD1002900D0B5E0089BA3
:1059A00012AA013B9B00D358002B00D084E20122B5
:1059B0000D9B043B596801320029FAD005990B0070
:1059C0008C46013362440792934242DC0E9A94461D
:1059D000A99A634492460B9A9B00944626AA904645
:1059E0009A44059B0A9A6344DB0098440C9B9446B6
:1059F0009946079BE144DB006344059353461868CE
:105A000002F090FE434618605960009B002B23DB98
:105A1000444600260027029D2268636803CD02F0F9
:105A20007DF802000B003000390001F03DFC083C1D
:105A300006000F005D45EFD14B469E60DF600423FA
:105A40009C460433E2449C46059BE144E04499456E
:105A5000D4D1079B0593B4E600260027ECE732007B
:105A60003B000020864902F0D3FA06000F00002C0C
:105A700000D175E7069A0020814900F0ABFB0200D7
:105A80000B003000390002F0C3FA06000F0067E790
:105A9000069B002B12D1059B12AA013B9B00D558F7
:105AA000EB1507930DE7059B12A95A1E920012AB46
:105AB0009B5810935B025B0A8B504EE70022714BA0
:105AC00001F060FA00280ED10023079348E75346FF
:105AD00000260027C0C39A4608239C46E144DA45C5
:105AE00000D03AE659E601239C4601330793059B13
:105AF000E044002B00DDEEE632003B000020604970
:105B000002F086FA06000F002AE743460B93069B35
:105B100012A8183B190006939300C3580092002B5B
:105B20000FD156481300844612A8634484469B0054
:105B30006344043B5868013A18390028F9D00092B0
:105B40000691069A00204E4900F044FB009B040099
:105B50000D00002B00DAB3E112AA94469F00DB008F
:105B600067449C460A9A0593624493461600386837
:105B700002F0D8FD22002B0001F0D0FF424B306034
:105B8000716000222000290001F0C8FF083E74ABBC
:105B900004000D00043FB342E9D100239A464EAB06
:105BA0000293089B99464B4600260027002B21DBD9
:105BB0008020364B5D469846C005354900260027B3
:105BC000002408E008239C460835E044A24511DB88
:105BD0004346186859682A686B6801F09FFF020005
:105BE0000B003000390001F05FFB013406000F00AC
:105BF000A145E7DA029A53469446DB0063441E60EF
:105C00005F6001239C46093BE2449C4674ABE3443D
:105C10009B45C8D1029B9946A89B022B00DD82E0E0
:105C2000002B37DC1DD1059B00254B441E000024B2
:105C3000326873682800210001F036FB009B0500E4
:105C40000C00083E5A1E0092F2D2079B002B03D094
:105C500080231B069C4664442A00230009990A609D
:105C60004B6007200B9B18409F239B009D443CBC2E
:105C700090469946A246AB46F0BDC046FFFFFF3FA7
:105C80000000F03F0000E03F0000703EA8AB0000C5
:105C9000FB21F93F059B00204B441E0000214CAF27
:105CA00032687368083E01F0FFFABE42F8D1079BE4
:105CB000002B24D08023099A1B06CB181060536058
:105CC0000B0002004E984F9902F0A2F9009B002BA6
:105CD0000BDD012450AD0CCD01F0E6FA009B013440
:105CE000A342F8DA079B002B03D080231B069C46B7
:105CF00061440B00020009998A60CB60B1E70200A1
:105D00000B00099C226063600B0002004E984F99C3
:105D100002F07EF9009B002BDBDC0B0002000999EE
:105D20008A60CB609DE7A89B032B9AD1009B002B38
:105D300000DCE3E07E4A059B94464B441E685F68A6
:105D4000009B63449A46DB004B4498464CAB9B4611
:105D500043465C681B681800210032003B0002903B
:105D6000039101F0A1FA04000D0002000B0002985B
:105D7000039902F04DF93B00320001F095FA4346D9
:105D80009860D9601C605D6008235B429C46E044DB
:105D900026002F00C345DBD1009B012B00DCADE0CA
:105DA000059BC8464B441E685F685346DB009B4614
:105DB000D844434630005C681B6839000093019466
:105DC0001A00230001F070FA04000D0002000B001D
:105DD0000098019902F01CF93B00320001F064FACE
:105DE00043469860D9601C605D6008235B429C4616
:105DF000E04426002F00C145DBD15D46002700248A
:105E000008354D4450AE2A686B683800210001F017
:105E10004BFA083D07000C00AE42F4D1079B002B63
:105E200071D0099A4E994B461160802109068C4623
:105E30005B684946634453604B46DB68896863444A
:105E400064449160D360176154610AE79946434600
:105E50000B93069B30005A42390000F0BBF9002238
:105E6000344B04000D0001F08DF8002832D0324B85
:105E700000222000290001F051FE02F01DFC4A46DC
:105E80000600970002F04EFC00222A4B01F046FE6D
:105E900002000B002000290002F0BAF802F00CFC0E
:105EA00012AAD0514A46069B01321833009206933B
:105EB000930012AAD65044E601227FE500243AE579
:105EC000A89B022B14DC002B0FDC00D0C9E60025B8
:105ED0000024BAE64B46200029009E0002F0ECFBAD
:105EE00012AB98514B4600932BE600200021DEE6D2
:105EF0004EAB9946A89B032B00D0B2E6079B002728
:105F00000024002B8DD14E9A4F9B09990A604B605B
:105F10004B469A68DB68009201938A60CB603A0036
:105F200023000A614B619CE676AB0A9335E4C046D8
:105F3000FFFFFF1F000070410000703EF0B54F46AC
:105F40004646C0B487B000920193464A4B00814652
:105F500088465B08934205DC02F0AEFB4146031E17
:105F6000484666D04A4643464846414601F0D6FD7B
:105F700004000D0002000B004846414601F0CEFD32
:105F8000394A3A4B06000F002000290001F0C6FDF7
:105F9000374A384B02F03CF822002B0001F0BEFDDE
:105FA000354A364B01F080F922002B0001F0B6FD96
:105FB000334A344B02F02CF822002B0001F0AEFDE6
:105FC000314B324A01F070F90E9B02900391002B85
:105FD00034D00098019900222D4B01F09FFD029AC8
:105FE000039B049005913000390001F097FD0200F9
:105FF0000B000498059902F00BF822002B0001F029
:106000008DFD009A019B02F003F8224A04000D0066
:10601000214B3000390001F081FD02000B0020000F
:10602000290001F041F902000B004846414601F009
:10603000EFFF07B00CBC90469946F0BD02000B0084
:106040002000290001F06AFD124A134B01F0E0FF25
:1060500032003B0001F062FD4A46434601F024F95C
:10606000E7E7C046FFFF3F3E7CD5CF5A3AD9E53D32
:10607000EB9C2B8AE6E55A3E7DFEB157E31DC73EF9
:10608000D561C119A0012A3F1111813FA6F8101155
:106090000000E03F495555555555C53F49004B084F
:1060A00019007047454AF8B5564692464B005B0DBD
:1060B0009A444D465F4644465246F0B48946050030
:1060C0000C000E000700132A22DC002A47DB524690
:1060D0003B4B134198460B0042461340034311D0FB
:1060E000384A394B01F0E0F80022002300F040FF6D
:1060F000002805D0002C41DB4E46434600279E4336
:10610000380031003CBC90469946A246AB46F8BDEB
:106110005246332A08DD8023DB009A45F2D1020083
:106120000B0001F0C1F8EDE7284A944601226344D0
:106130005242DA4093460242E4D0224A224B01F016
:10614000B3F80022002300F013FF0028D8D0002C61
:106150001ADB5B464E469F4338003100D2E7194AAE
:10616000194B01F0A1F80022002300F001FF0028E4
:10617000C6D0002C16DB00270026C1E7802352463C
:106180005B0313419944B7E75346142B12D03423D1
:10619000524601279B1A9F407F19AF429B415B42A9
:1061A0009944D6E76400640825430027002DA7D052
:1061B000074EA5E7133B9C46E144CAE701FCFFFFFD
:1061C000FFFF0F009C7500883CE4377EEDFBFFFF6E
:1061D0000000F0BF4B0070B55B0D14000A00002BEF
:1061E0001AD14B005B08034315D00022224B01F06B
:1061F00095FC224B0A009C4222DB4B005B0D363B98
:106200001F4DE318AB4220DC002B0DDD1D4C1B05A0
:1062100022401A43110070BD1B4DAB42F0D1020069
:106220000B0001F041F8F6E71D00353518DA174B81
:1062300002009C420ADC0B001548164900F032F8B7
:10624000134A144B01F06AFCE5E702000B00124808
:10625000124900F027F8104A104B01F05FFCDAE712
:10626000084C363322401B051343190000220C4B07
:1062700001F054FCCFE7C04600005043B03CFFFFA4
:10628000FE070000FFFF0F80FF07000050C3000063
:1062900059F3F8C21F6EA5019C7500883CE4377E57
:1062A0000000903C30B54A00DB0FDB0752081A4370
:1062B000110030BD03210A4802680A430260094800
:1062C00002680A4302600849084A094B9B1A03DD29
:1062D000043BC858D050FBDC00F0B4F9F9F74AFF92
:1062E00024050040540500407CAE00000000002062
:1062F00038020020FEE7FEE7FEE7FEE7FEE7FEE7E6
:10630000014B18607047C04674010020F7B50023A8
:10631000202877D83C4B8000C258042A14D006D8D5
:10632000022A0DD00ED80423012A14D069E0062ACF
:106330000ED00BD31A2A0DD002231B2A0BD060E0FB
:10634000082308E0102306E0202304E0402302E0B5
:10635000802300E001232D4A1268082A04D9092A63
:1063600005D00A21022404E00821002401E01100E4
:106370000124A02501261C272548ED004651254D66
:10638000254E2D681B02AD003D400195234D2D6823
:1063900000958559AC466746214D3D401D438551CA
:1063A0008359C0259C46009BAD021D40FF236746D4
:1063B0001B023B402B43019D1D43009B5F0160235B
:1063C0001F402B003B431C4301238451154C0360A9
:1063D00063680F48002BFBD00024124B01255C6042
:1063E000A123DB00C3584560A025ED0044511BB23A
:1063F000914207D002D98A1AD34003E0521A93403F
:1064000000E000231800FEBD7CA9000078010020F8
:106410000070004070010020040500006C010020A5
:10642000FF00FFFFFC700040F0B520286CD8374B10
:106430008000C258364B1E68002E2ED1C22435482B
:10644000A4000759344B03253B40C0273F023B4380
:1064500003518023893C9B00FF3C03512F4F036075
:106460002F4B803CD859FF3CA043D8510437D85912
:10647000A8432043D8510837D8590C35A843083DC4
:106480002843D851A820C0001E508026C120760283
:1064900080001E501C601E4B1C60002314262148E7
:1064A00034005C43255804006F1C0FD1142058435E
:1064B0002250A0200325C132FF329200C0051550A2
:1064C000194A08001268082A03D10BE0AA4218D121
:1064D000ECE7082A02D9083AD14002E00820821AE3
:1064E0009140080014225343E3189A680C49513232
:1064F000FF32920058605050DA68C1239B00CA50A6
:1065000002E00133032BCBD1F0BDC0467CA90000D3
:106510008011002000E100E0FF00FFFF0405000003
:10652000009000407C010020740100201E4BF0B55B
:10653000596C18001D4A002914D0A025A12600235B
:106540000124ED05F600D1584F1C06D0D7187F68FE
:10655000002F02D027008F40AF5114333C2BF2D1D3
:1065600000234364131DA0254032944600200124DB
:106570000F4EED05DA680F49920057180A49521874
:10658000526C002A0CD01A1F1268511C05D01968D1
:10659000FF2902D021009140A9513A00FC325064F9
:1065A00014339C45E6D1F0BDFC9000407C010020F6
:1065B0000C0500000090004000B5202816D80C4AB9
:1065C00083009B58032911D8A0220800C133FF3350
:1065D000D2059B0000F014FB02080406002104E031
:1065E0000C2102E0042100E00321D15000BDC0468F
:1065F0007CA9000020280DD8074B8000C058A0229D
:106600000123D2058340002901D1044901E0A121E1
:10661000C90053507047C0467CA900000C0500001B
:1066200003000020202B0AD8A222A021D200C905F5
:106630008858034A9B009B58D84001231840704754
:106640007CA900002D4B10B51A78012A19D12C4ACB
:106650001268120715D12B4AE0241168F0220800B5
:10666000104021420BD128490968114209D127491C
:10667000274A11608021274A0902116001E0302871
:10668000F1D01A78012A0DD11D490968090709D1ED
:10669000F0201C4909680140402903D11A490968C2
:1066A000014223D01B68DBB2012B25D1144B1B68A0
:1066B0001B0721D1134B1A68F0231A40A02A04D1DA
:1066C000114A12681A4203D016E0D02A14D1F7E713
:1066D000114B1A68012A03D1C022104B1A600BE03B
:1066E0000F4A1A601A68012AFCD1F5E7C1218020FF
:1066F000C900C0054250D5E710BDC046E00F00F00C
:10670000E40F00F0E80F00F0EC0F00F0DFFF07C02F
:1067100004050040186C004000EC064014EC0640F4
:1067200075930000F7B506000D000C008B1801935F
:10673000019B671B9C4207D0336821781B6830009F
:10674000984701340028F3D13800FEBD70B505002C
:106750000C00081E07D002F04FFD2B6802005B689A
:1067600021002800984770BD10B5FFF7EFFF10BD5E
:1067700010B540220021040002F011F9002320008E
:106780002364636410BD3F23026C10B5541C234086
:10679000446C9C4201D08154036410BD0023036407
:1067A00043647047436C026C934206D03F21C25C45
:1067B00001330B404364100001E001204042704768
:1067C000036C406C181A00D540307047436C026C63
:1067D000934201D0C05C01E0012040427047036C4D
:1067E000406C5A1C3F231340181A42424241D0B217
:1067F00070470120704710B503681322DB69984782
:1068000010BD70470369054A9950FC331A6A002A83
:10681000FCD0002201201A627047C0461C0500000F
:10682000030010B55C331A781F23134001221100B6
:1068300099400D4B0424D967C221036989005C503B
:106840005A60DA60A0220021D20099500122074943
:1068500052425A50064914305A500C395A50083195
:106860005A50FFF79BFF10BD04E100E00C0500004B
:106870001405000010B51430FFF7A2FF10BD10B5CD
:106880001430FFF7A3FF10BD10B51430FFF78AFFD7
:1068900010BD0000030070B55E331C780269604BC8
:1068A000D45003005D331C785E4BD4500300613339
:1068B0001C785D4B012C0CD105005F352E78A2258C
:1068C000ED005651050060352E78A125ED0056519A
:1068D00000E00024D4509623DB00994238D9962357
:1068E0001B01994237D996235B01994236D99623E9
:1068F0009B01994234D9E1239B01994232D99623D5
:10690000DB01994231D9E123DB0199422FD996234A
:106910001B0299422DD9E1231B0299422BD99623C0
:106920005B02994229D9E1235B02994227D9E123ED
:106930009B02994225D93D4B994224D9E123DB02A0
:10694000994223D9E1231B03994221D8384B21E0F6
:106950009E23DB021EE09D231B031BE0354B19E049
:10696000354B17E0EC239B0314E0344B12E0344B1F
:1069700010E0344B0EE0344B0CE0344B0AE0344B67
:1069800008E0344B06E08023DB0403E0324B01E0F7
:1069900080235B053149002453500423243953508C
:1069A0001100FC31CC600C62C121013489001460FB
:1069B0005C309460535003781F202200D9B2084005
:1069C000824080342648FF345BB20251002B13DA38
:1069D0000F230B40083B234C9B089B001B190324EF
:1069E0002140A140FC348C40DD69A543C0248C408B
:1069F00021002943D96111E0194C9B089B001B1908
:106A000003242140A140C025FC348C40AD005E59D8
:106A1000A643C0248C40210031435951026070BD0F
:106A20000C050000140500006C05000090D0030068
:106A300000D0BE0E00B013000050270000A04E0092
:106A400000F0750000509D0000F0EB0000903A014E
:106A500000E0D70100B0AF0300705F07240500001D
:106A600000E100E000ED00E0F7B5009308AB1B7813
:106A700000250193FA2304009B0083600E4B4560C0
:106A80000833036014300F001600FFF771FE230077
:106A90005C3327611E70009B084A9B0099582300B5
:106AA0005D331970019B20009B009A5823005E33D0
:106AB000DD701A70FEBDC046E8AB00007CA9000086
:106AC000036910B51A00FC32D2680400002A0AD00B
:106AD000A322D20099581430C9B2FFF754FE002205
:106AE0002369FC33DA6010BD10B50248FFF7E8FFF8
:106AF00010BDC04684110020162307B50222009362
:106B00000249013B0248FFF7AFFF07BD00200040EC
:106B1000841100207047000010B500F047F8FFF71F
:106B2000F9FF012000F024F8FDF760FFFDF772FF88
:106B3000024B002BFAD000E000BFF7E70000000096
:106B4000084A0949094B10B51B688858FA22190AE6
:106B50001B0618439200002300F01EFA4904C00BE4
:106B6000084310BD0405000000100140E81100209A
:106B700070B5041E09D0FFF7E3FF050000F014F81C
:106B8000FFF7DEFF401B8442F8D870BD0022044BA3
:106B90009A60044A13680133DBB213607047C04641
:106BA000FC100140E811002070470000C421114A88
:106BB00089005058104B0340C0200002034353503B
:106BC000802391399B02FF39535013608023A32205
:106BD0000021DB05D20099500122A1209A60074BC9
:106BE000C0001950C12002318000195040301950A6
:106BF0001A60704700E100E0FF00FFFF0010014055
:106C000002B4714649084900095C49008E4402BC3F
:106C10007047C046002243088B4274D303098B425D
:106C20005FD3030A8B4244D3030B8B4228D3030C5C
:106C30008B420DD3FF22090212BA030C8B4202D3FE
:106C40001212090265D0030B8B4219D300E0090A26
:106C5000C30B8B4201D3CB03C01A5241830B8B422F
:106C600001D38B03C01A5241430B8B4201D34B0318
:106C7000C01A5241030B8B4201D30B03C01A52417D
:106C8000C30A8B4201D3CB02C01A5241830A8B4202
:106C900001D38B02C01A5241430A8B4201D34B02EB
:106CA000C01A5241030A8B4201D30B02C01A52414F
:106CB000CDD2C3098B4201D3CB01C01A5241830903
:106CC0008B4201D38B01C01A524143098B4201D33D
:106CD0004B01C01A524103098B4201D30B01C01A68
:106CE0005241C3088B4201D3CB00C01A52418308E2
:106CF0008B4201D38B00C01A524143088B4201D30F
:106D00004B00C01A5241411A00D20146524110466E
:106D10007047FFE701B5002000F0F0F802BDC04663
:106D20000029F7D076E7704703460B437FD4002253
:106D300043088B4274D303098B425FD3030A8B420F
:106D400044D3030B8B4228D3030C8B420DD3FF2279
:106D5000090212BA030C8B4202D31212090265D047
:106D6000030B8B4219D300E0090AC30B8B4201D3FA
:106D7000CB03C01A5241830B8B4201D38B03C01A41
:106D80005241430B8B4201D34B03C01A5241030BB8
:106D90008B4201D30B03C01A5241C30A8B4201D369
:106DA000CB02C01A5241830A8B4201D38B02C01A14
:106DB0005241430A8B4201D34B02C01A5241030A8B
:106DC0008B4201D30B02C01A5241CDD2C3098B4270
:106DD00001D3CB01C01A524183098B4201D38B01ED
:106DE000C01A524143098B4201D34B01C01A524190
:106DF00003098B4201D30B01C01A5241C3088B42D5
:106E000001D3CB00C01A524183088B4201D38B00BF
:106E1000C01A524143088B4201D34B00C01A524161
:106E2000411A00D201465241104670475DE0CA0F38
:106E300000D04942031000D34042534000229C46F8
:106E400003098B422DD3030A8B4212D3FC22890102
:106E500012BA030A8B420CD3890192118B4208D3D8
:106E6000890192118B4204D389013AD0921100E03A
:106E70008909C3098B4201D3CB01C01A524183094E
:106E80008B4201D38B01C01A524143098B4201D37B
:106E90004B01C01A524103098B4201D30B01C01AA6
:106EA0005241C3088B4201D3CB00C01A5241830820
:106EB0008B4201D38B00C01A5241D9D243088B4276
:106EC00001D34B00C01A5241411A00D20146634619
:106ED00052415B10104601D34042002B00D549427D
:106EE000704763465B1000D3404201B5002000F0BC
:106EF00005F802BD0029F8D016E770477047C04674
:106F0000D0400B1C1141203A03D49C461341184336
:106F100063465242934018437047C0468446101C53
:106F200062468C46191C634600E0C0461FB500F05F
:106F30008BFD002801D40021C8421FBD10B500F010
:106F4000DFFC4042013010BD10B500F07DFD00288F
:106F500001DB002010BD012010BDC04610B500F0BF
:106F600073FD002801DD002010BD012010BDC046CA
:106F700010B500F005FD002801DC002010BD012047
:106F800010BDC04610B500F0FBFC002801DA00205F
:106F900010BD012010BDC046F0B54F464646C0B4F6
:106FA0001604360C9946330005042C0C070C150CFE
:106FB00063437E436F4365431C0CAD1964199C46C3
:106FC000A64203D980235B02984647446346250CBA
:106FD000EF191D044B464A4343432D0C2404641906
:106FE0009918C91920000CBC90469946F0BDC046BE
:106FF000F0B557464E4645464300E0B44602884643
:10700000760A1F0EC40F002F47D0FF2F25D0002374
:1070100080259A469946F600ED042E437F3F43466D
:1070200042465D02D20F5B006D0A1B0E904640D0B7
:10703000FF2B39D080220020ED00D20415437F3B86
:10704000FB1842465746591C62408C4607430F2F97
:107050005CD86F49BF00C9598F46002E45D108231F
:107060009A46063B9946DAE7424602282DD0032885
:1070700000D1C3E0012800D0A2E000250026024094
:10708000D4B27602ED05760A2E43E407264330009B
:107090001CBC90469946A246F0BD002E1AD104238E
:1070A0009A46033B9946BAE72A00511E8A41901C32
:1070B000C6E70120002DC3D0280001F0C9FB431F03
:1070C00076309D4043420020BAE70124FF2514405A
:1070D0000026D6E7300001F0BBFB431F9E40002393
:1070E000763047429A46994699E70C239A46093BDF
:1070F000994694E780260024F603FF25C1E7350072
:107100004846B2E7350022004846AEE72904090C9C
:107110000800370C3604360C2C0C79437043674357
:107120007443060C64183619B14203D98021490210
:10713000884647440004000C310409188D01681E7C
:107140008541890E2943350CED19AD010D43290107
:1071500004D5012369081D4063460D4319007F31A2
:10716000002925DD680704D00F202840042800D01E
:107170000435280103D5274980330D401900FE2925
:10718000A3DC0124AD016E0A1440CDB279E7802062
:10719000C003064207D0054205D128434602760ABD
:1071A0004446FF256DE706437602760AFF2568E729
:1071B0000124611A1B2905DD14400025002660E723
:1071C0006346CBE72E002023CE40591A8D406B1E1C
:1071D0009D412E43730704D00F233340042B00D06E
:1071E0000436730104D5012401251440002648E724
:1071F0000124B601760A1440002542E780260124C6
:10720000F6032E437602760A1440FF2539E7C0467E
:1072100018AC0000FFFFFFF770B5002830D0C3178F
:10722000C5185D40C40F280001F012FB9E231B1AF5
:10723000962B0DDC9622D21A95406A02520AD8B2D9
:107240005202C005520AE40702432243100070BDF7
:10725000992B19DC9922D21A9540124A2A406907C3
:1072600004D00F210D40042D00D00432510103D56C
:107270000C4B1A409F231B1A9201520AD8B2DFE727
:10728000002400200022DBE705222E00121AB9217B
:10729000D6402A00C91A8A40551EAA413500154316
:1072A000DBE7C046FFFFFFFBF8B556465F464D469D
:1072B0004446F0B40F00FD0FAA4609037C002E00DF
:1072C0005F00450F490A7F0D2943C5001803BC46DE
:1072D000400A570F640DDB0F3843D2009A4500D1A6
:1072E000AAE06646A61B002E00DCFFE06346002BEA
:1072F00039D10300134300D0D9E06B0709D00F2325
:107300002B40042B05D02B1DAB42AD416D424919DA
:107310001D000B0200D482E0CA4B01349C4200D114
:10732000FEE00A005646C84BED081A4050076405B7
:1073300052020543120B640D002112030B0D1B05B5
:107340006405120B1A436308C04CF60714401C4333
:10735000640064083443280021003CBC90469946F0
:10736000A246AB46F8BDB74B9C42C6D080231B0457
:107370001843382E00DDEBE01F2E00DD1EE1202338
:107380009B1B9C4603006746BB409846130047463C
:10739000F3403B436746BA40571EBA4113430200CD
:1073A000F240EB1A9D42B6411D008A1A7642911BAB
:1073B0000B0231D54A02560A002E00D1B4E030004B
:1073C00001F046FA0300083B1F2B00DDB5E0202248
:1073D0002900D21AD1409E400A009D4032439C426F
:1073E00000DDB1E01C1B631C1F2B00DDD5E020215C
:1073F00014002800C91A8C40D8408D400443DA405C
:10740000681E854111002543002476E7414631433B
:1074100000D134E2310045466B0700D06FE7564695
:107420004807ED08C9080543864B9C4235D00A033E
:107430006405120B640D7FE76346E31A9B46002B3D
:1074400000DC8BE06746002F3CD07E4FBC4200D171
:1074500053E780273F0438435B46382B00DCF7E0D6
:107460000243501E82410020D2B253194218AB424F
:1074700089411D00494289180B02CDD5714B013459
:107480009C4200D13DE101206F4A6B080A40284030
:107490001843D507054351082FE72B000B4300D1B4
:1074A000CBE180231B030B431A03120B44E7013E7D
:1074B000002E6DD1AE1AB5429B41091A5B42C91A22
:1074C000350075E70700174300D116E701235B423B
:1074D0009C46E3445B46002B00D0E0E0AA18AA4299
:1074E0009B4109185B4259181500C5E7002E75D15C
:1074F000661C7605760D012E00DCF3E0AE1AB04670
:107500004545BF410E1A7F42F61B370200D48FE07B
:10751000551BAA42B641411A76428E1B9A464BE74A
:1075200056460022002507E7280001F091F9203097
:107530000300083B1F2B00DC49E72A002838824063
:1075400000259C4200DC4DE73F49E41A1140D4E697
:107550000243501E8241D3B2002222E7002B00D00A
:10756000F3E0631C9C465B055B0D012B00DC9FE098
:10757000344B9C4500D1C3E0AA180918AA428041A7
:1075800040424118CD075208154349086446B4E605
:107590002C4B9C4200D0ECE6AFE611001F3CE140D2
:1075A0000C00202B00D17FE04021CB1A9A401543DC
:1075B0006A1E95410021254300242DE73300070072
:1075C000203BDF403B00202E70D04027BE1BB04048
:1075D0000243501E824113430022E2E6002C4FD0AA
:1075E000184CA44500D1ABE080242404764221430A
:1075F000382E00DDDFE01F2E00DD43E12027BC1B1D
:10760000A1460C004F46BC40A0462C004746F44023
:107610003C434F46BD406F1EBD41F1402C43151BFE
:10762000AA429241411A5242891A64469A46BFE6DA
:1076300041464546314300D0BEE6002600240025E1
:10764000F2E6C046FF070000FFFF7FFFFFFF0F804D
:107650001F2B59DC2027FF1ABC46070063469F40BA
:107660005B46B9461700DF40B8464F4643461F43C6
:1076700063469A40531E9A415B463A43D840F4E62B
:107680000C002C435CD0F643002E55D1551BAA426A
:10769000A441411A6442091B9A46644688E6964F03
:1076A000BC4200D0D8E628E6002280E700208FE721
:1076B0000B002B43002C00D0C2E0002B00D101E1D5
:1076C0000300134300D118E6AB18AB42B6410918CA
:1076D000764271180A0200D409E1884A1D0011405F
:1076E00064460AE6002C5BD10E002E4300D08AE0EF
:1076F0000100114300D1C2E0010015009A46FCE5EB
:107700006446002100258FE620235B429C46DC4432
:1077100063460700DF405B46BC46202B00D1ACE04F
:1077200040235F46DB1B98400243501E8241634664
:1077300013431A00002098E66F4CA44500D057E789
:107740000100150064469A46D7E5002C39D10C009B
:107750002C436ED0DB43002B1AD0674CA44568D075
:10776000382B00DDA4E01F2B00DDAEE020240F004D
:10777000E41AA740B9462F00DF40B846A3464F465B
:10778000444627435C46A5406C1EA541D9403D4375
:10779000AD1895429B4109185B42591864466BE647
:1077A0000C002C4315D1010011437BD001001500C2
:1077B0009A46514CA1E50D43691E8D410021ECB262
:1077C0002DE74D4CA44534D0802424045B42214352
:1077D000C6E7040014434ED0ED084C072C43802527
:1077E000C9082D03294208D0C6082E4205D1D20867
:1077F000410711430C009A463100620FC900E500B1
:1078000011433D4C79E50600164300D175E5AE1AEB
:10781000B0464545BF410E1A7F42F61B370200D4E1
:10782000F4E5551BAA42B641411A7642891B9A4695
:1078300063E50100150064465FE5002200257BE555
:10784000002B3BD00300134315D0ED084B072B430F
:107850008025C9082D03294207D0C4082C4204D131
:1078600041070B002100D2081343C9005A0F1143EE
:10787000DD00214C41E5204C3FE5002054E7002687
:107880000025D1E534000F00203CE7403C00202ECD
:107890002BD04027BE1BB1400D43691E8D410021F6
:1078A0002C43BCE6802100260903134C0025BBE5D0
:1078B0000D43691E8D410021EDB269E701001500FD
:1078C0000D4C1AE50100150017E51C000F00203CC7
:1078D000E7403C00202B0CD04027FB1A99400D4379
:1078E000691E8D410021254352E70021D4E71D0088
:1078F00092E50021F3E7C046FF070000FFFF7FFF8E
:10790000F0B55F4656464D464446F0B41F035C0052
:10791000DB0F9A46194B0E034D00C90F8046360BFC
:107920006D0D8B4691463F0B640D9D4219D0134B54
:107930009C421BD00123A54206D018003CBC9046B7
:107940009946A246AB46F0BDBE42F6D1C845F4D139
:10795000D34510D0002DF0D1304303005A1E93417F
:10796000EBE7310001230143E7D1E0E73A4301238C
:10797000002AE2D1DEE70023DFE7C046FF07000070
:10798000F0B55F46444656464D46F0B41F033C0BE7
:107990002C4F0E034D00A3465C008446360B6D0D44
:1079A000C90F9046640DDB0FBD422BD0254FBC4262
:1079B0002ED0002D0ED13043070081467842784109
:1079C000002C17D15F463A4314D14B460020002BC0
:1079D0000AD006E0002C02D15846024301D0994259
:1079E0001AD00123484218433CBC90469946A2460F
:1079F000AB46F0BD0028F2D0584258410122404227
:107A00001043F1E737000743D0D002204042EBE7B4
:107A10005F461743CDD0F8E7A542E2DC05DB5E45C3
:107A2000DFD808D000205E45DED24842484101231D
:107A300040421843D8E7C445D3D80020C445F4D306
:107A4000D2E7C046FF070000F0B55F464D4644460A
:107A50005646F0B41C03240BA4462F4C0F034D00D4
:107A60005E00C90F80463F0B6D0D8B469146760D2B
:107A7000DB0FA54220D0284CA64222D0002D12D1E7
:107A8000384344424441002E20D0002C0DD05C42AB
:107A9000634101245B421C4320003CBC9046994654
:107AA000A246AB46F0BD002E17D05B4519D05B4611
:107AB0005C4201231C43EFE7390002240143EBD170
:107AC000D9E7614602241143E6D1D7E761460A436C
:107AD000DBD100240028DFD0E9E761460A43E4D186
:107AE000E5E7B54203DD01225C421443D4E7B54229
:107AF000CDDB6745DBD809D000246745CCD2594699
:107B00004C426141012449420C43C5E7C845CED8E7
:107B10000024C845F3D3BFE7FF070000F0B55F4678
:107B200056464D464446F0B40D0399464E002B0B85
:107B300087B00700924680469B46760DCC0F002EFC
:107B400069D06D4B9E4235D05B468022DD00120429
:107B5000430F13432B439B46C3009846674B0027B4
:107B60009C460023664401934A4615035000D20FF9
:107B700053462D0B400D914600D176E05E4A90426F
:107B80006CD080225B0F120413435C4AED009446D4
:107B90001D4353460022DB00604449463618701CE2
:107BA0006140029017430F2F00D9AFE05448BF0047
:107BB000C759BF465B461F4300D088E000239B4661
:107BC0009846023308270193CEE74946022A6AD035
:107BD000032A00D109E2012A00D0BBE111400022B2
:107BE000002300259046CCB200212D030A0D12057A
:107BF0002D0B1543434A1B0515401D436D00E4073B
:107C00006D0825434046290007B03CBC9046994684
:107C1000A246AB46F0BD034352D05B46002B00D1D9
:107C20008AE1584600F014FE03000B3B1C2B00DDDC
:107C30007BE11D22D31A3A0001005D46DA40083983
:107C40008D4013008F402B439B46B8462E4B002798
:107C50009C46002360444642019385E752462A43EE
:107C60002CD100250023022297E752462A4321D037
:107C7000002D00D154E1280000F0EAFD03000B3B89
:107C80001C2B00DD46E11D21CB1A51460200D940D4
:107C90005346083A954093400D431B4A944660442E
:107CA0004042002279E7012400220C40124B0025BB
:107CB000904699E70025002301226EE703226CE736
:107CC00000239B4698460133042701934CE7032386
:107CD0000C27019348E700238025984600242D03B4
:107CE000054B81E75D464346019A6FE75D46434693
:107CF0002100019A6AE7C046FF07000001FCFFFF70
:107D000058AC0000FFFF0F80F30300004246120C46
:107D100091461A0C9446424617044A461B041B0C13
:107D20005A43604690464A464243100003926246D8
:107D30001C003F0C7A437C4342440192220C924641
:107D4000019A5244904506D98246802040028046DE
:107D5000C24450460390100C049048462404240C5E
:107D60001204121905922A0C2D042D0C68432C00C4
:107D7000824648467C4350438146200C8046574308
:107D800057444744BA4503D9802040028046C14445
:107D9000380C3F04B84648442404240C019004984D
:107DA000A044404404905846000C814658460404C0
:107DB000200C8246070048465F434C4643436046DA
:107DC00060436446834650464443380C8446E41876
:107DD0006444A34203D980235B029C46E3444846A3
:107DE0003F04230C3F0C2404E419574668436F43B7
:107DF00084464D46504655434243380C81466244C2
:107E00004A445B44944503D980204002844665443B
:107E100003983F04834604983F0C8446E344C345DB
:107E2000804140428246100484460198674484465B
:107E30006744A344BC46A345A4419946D444644244
:107E40008742BF41D4458041E144A04699459B41CA
:107E50007F424042C8440743120CBA18A045A441CF
:107E60005F423B0064422343D71843467D19DB0D34
:107E70006D021D435B465A02059B1A43531E9A41ED
:107E80005B46DB0D1A4343465B021343EA0107D509
:107E900001225C0813402343EA07029E13436D0846
:107EA000574AB218002A4BDD580709D00F20184056
:107EB000042805D0181D98429B415B42ED18030031
:107EC000E80104D54F4A15408022D200B2184E482E
:107ED000824200DDE7E60124DB08680718436D02F3
:107EE000530580462D0B5B0D0C407DE680225946E4
:107EF0001203114208D0154206D115432D039846AE
:107F00002D0B4C46414B6FE65D4615432D032D0B63
:107F10003E4B69E603005546283B9D400023BCE6E6
:107F2000504600F095FC2030A8E60300283B9F4017
:107F30000023BB46984689E600F08AFC203073E6B1
:107F40000124A61A382E07DD00220C40002300254C
:107F5000904649E6029EA3E71F2E20DC20222C003B
:107F60001800921BF040944093400443581E8341F4
:107F70001C43F540630709D00F232340042B05D091
:107F800023001C1D9C4292415242AD182B021FD56A
:107F9000012400220C4001230025904624E61F20E6
:107FA0002C004042821AD440202E1CD04022961B26
:107FB000B5402B43581E834107202343184000251A
:107FC000002809D00F2200251A401C00042AD8D10D
:107FD000230068076D022D0B0124DB08034398463C
:107FE0000C40002300E60025E3E780220124120371
:107FF00015432D0398462D0B0C40044BF4E5C04669
:10800000FF030000FFFFFFFEFE070000FF07000068
:10801000F0B557464E464546E0B40E001100F20F4B
:108020009246C500420F180337037400400A4E0FF2
:108030007F0A3043CF4E17435A00640D520DDB0FB9
:10804000C900B24200D1E5E001267340A61AB44649
:10805000534500D1AFE0002E00DC0DE1002A3AD1FB
:1080600003000B4300D0E4E06B0709D00F232B4043
:10807000042B05D02B1DAB42AD416D427F191D0075
:108080003B0200D488E0BB4B01349C4200D110E19C
:108090003A00B94B51461A4001235007ED085202ED
:1080A00064050543120B640D0B40002128001203E8
:1080B0000D0D120B64052D0515436208AF4CDB074F
:1080C0002C401443640064081C4321001CBC9046EF
:1080D0009946A246F0BDA74B9C42C5D080231B0405
:1080E00018436346382B00DDFDE01F2B00DD30E137
:1080F000624620239B1A02009A40664690460A0078
:108100009940F24046464B1E994132431143634623
:108110000200DA40691A8D429B410D00BA1A5B4297
:10812000D71A3B0235D57A02530A98464346002BAC
:1081300000D1C4E0404600F08BFB0300083B1F2B3E
:1081400000DDC5E020222900D21A4746D1409F40D9
:108150000A009D403A439C4200DDC0E01C1B631CAA
:108160001F2B00DDE4E0202114002800C91AD840AC
:108170008C408D400443DA40681E8541170025433A
:10818000002471E7424663461A4300D14CE2674639
:1081900045466B0700D069E7012351467807ED0893
:1081A000FA080B40054373498C4238D0120364052A
:1081B000120B640D79E7002E00DC9AE0002A47D00C
:1081C0006C4A944200D14FE7802212041043624669
:1081D000382A00DC08E10143481E81410022C9B26F
:1081E0004919D219A942BF410D007F42BF183A0276
:1081F00000D442E15F4A0134944200D14EE10120B3
:108200005D4A69083A4028400843D50705435708A6
:108210009A4629E706000E4300D017E714E7290025
:10822000114300D1F9E1802109030A431203120B23
:108230003BE701235B429846C4446346002B72D15E
:10824000691A8D429B413F1A5B42FF1A0D0068E795
:1082500002000A4300D107E7012252429046C4447B
:108260006246002A00D0E6E06918A942B6413F18EC
:108270007642F7190D00BAE7002E00D080E0621CAC
:108280005205520D012A00DCF9E06A1A91464D456B
:10829000B6413A1A7642921B9046120200D499E0F7
:1082A0004D1BA9428941C71B49427A1A90469A46FA
:1082B0003CE752460123002513400022F5E6280042
:1082C00000F0C6FA20300300083B1F2B00DC39E722
:1082D0002A002838824000259C4200DC3EE7264FD9
:1082E000E41A1740C0E60143481E81410022C9B28A
:1082F00010E7002E00D0F1E0621C94465205520DAA
:10830000012A00DCA0E01B4A944500D1C5E06918B1
:10831000A94292413F185242D2194908D5070D434C
:1083200057086446A0E6134B9C4200D0D9E69BE672
:1083300011001F3CE1400C00202B00D180E04021C7
:10834000CB1A9A4015436A1E954100272543002405
:108350001FE763460200203BDA406346202B71D0C2
:10836000402366469B1B98400143481E81411143B0
:108370000022CFE6FF070000FFFF7FFFFFFF0F8017
:10838000002C48D0CA4CA24200D1A2E07442A146BF
:108390008024240427434C46382C00DDDBE01F2CCE
:1083A00000DD44E14E462024A41B3E00A640A24628
:1083B000B0464C462E00E640B44646466446264348
:1083C0005446A5406C1EA54134002C434D46EF4059
:1083D0000D1B28E04A4643464D461A4300D0A5E609
:1083E000002300240025DEE61F2A5ADC66462022F0
:1083F000921B060096409146B04662460E00D6405B
:10840000424616434A4691404A1E91410200604648
:108410003143C240E4E63C002C435AD0F443A14629
:10842000002C52D14D1BA9428941C71B49427F1ADA
:1084300014009A4675E69E4A944200D0C7E613E6B9
:1084400000227FE700208FE7002C00D0C8E03B002F
:108450002B4300D10FE103000B4300D104E6691860
:10846000A9429B413F185B42DF193B0200D41AE14D
:10847000904B0D001F406446F6E59A4689E63A00A7
:108480002A43002C5CD1002A75D102000A4300D196
:10849000CAE007000D009A46E6E564460022002582
:1084A00081E662460600203AD6406246B046202A5F
:1084B00000D1B7E040226646921B904001434246FD
:1084C000481E8141114300228AE6794CA24200D025
:1084D00061E707000D0014009A46C5E5002C41D164
:1084E0003C002C4378D0F443A146002C20D0704CA3
:1084F000A24271D04C46382C00DDB2E01F2C00DDCA
:10850000BCE02026341BA2463C005646B4404E46F2
:10851000A0462C00F440A446444666463443A44694
:108520005446A54064466E1EB54125434C46E7407F
:108530006D188D4289413F184942CF19140056E603
:10854000002A2FD102000A4300D184E007000D0069
:108550009A46574C88E53D436F1EBD41ECB200275B
:108560000D1B60E7524CA24236D07442802636047E
:10857000A1463743BEE702000A4300D174E56A1AF8
:1085800090464545B6413A1A7642921B94461202ED
:1085900000D4F7E54D1BA9428941C71B49427F1A08
:1085A0009A4661E502000A433AD0ED087C072C4365
:1085B0008025FA082D032A4208D0C7082F4205D18A
:1085C00045072C003A009A46C9080C43670FD200B1
:1085D000E5001743364C47E507000D00140043E55E
:1085E0003A002A4343D002000A4319D0ED087C0721
:1085F0002C438025FA082D032A4207D0C6082E42B4
:1086000004D147073C003200C9080C43D700620F71
:10861000E50017439A46264C26E50022002544E54E
:10862000234C21E5002049E700230025BBE54C460B
:108630003E00203CE6404C46B446202C31D040243D
:108640004E46A61BB7403D436C1EA54164462C43D5
:1086500000270D1BE7E6802200231203144C00259F
:10866000A1E53D436F1EBD410027EDB260E7070065
:108670000D000F4CF8E407000D00F5E44E463C00F9
:10868000203EF440A0464C46202C0ED040244E46BE
:10869000A41BA7403D436F1EBD4144460027254310
:1086A00046E70027CFE70D0073E50027F2E7C04655
:1086B000FF070000FFFF7FFF0B0330B5134D1A0BC0
:1086C0004B005B0DC90F0024AB4211DD104CA342DF
:1086D00010DC8024640322430E4CE41A1F2C0CDDB2
:1086E0000D48C31ADA4013005C42002900D11C0077
:1086F000200030BD094BCC18FAE7E040084CA446F6
:1087000063449A4013000343EEE7C046FE030000B3
:108710001D0400003304000013040000FFFFFF7F6E
:10872000EDFBFFFF70B5002830D0C317C4185C40C4
:10873000C50F200000F08CF8174B184A1B1AD21AEC
:108740001F2A18DD164AD21A9440002224035B0522
:10875000240B5B0D0021100024030A0D1205240BCD
:108760001443104A1B0514401C436400ED076408C1
:108770002C43210070BD210091400A000B21081AF2
:10878000C4405B052403240B5B0DE3E700250023B5
:1087900000240022DEE7C0461E040000330400006F
:1087A00013040000FFFF0F804200120E511C430211
:1087B000C9B270B55D0AC40F012915DDE021890039
:1087C0008C466D071B0B6244002128000D0D2D0502
:1087D0002B431C4D52052B40520813435B00E4070A
:1087E0005B082343190070BD002A15D1002D1FD04E
:1087F000280000F02DF80A281DDC0B232A001B1A84
:10880000DA4013000200153295400F4A1B03121A7A
:1088100052051B0B520DD7E7002D06D080221B0BF3
:10882000120313436D07094ACEE7084A0023CBE73A
:1088300000220023C8E703000B3B9D402B000025CE
:10884000E3E7C046FFFF0F8089030000FF07000039
:108850001C2101231B04984201D3000C10391B0A70
:10886000984201D3000A08391B09984201D3000934
:10887000043902A2105C40187047C046040302028B
:108880000101010100000000000000007FB51D0093
:108890000A4B06001B68D868002A02D1084C230046
:1088A00001E01300074C0293009133002A000649AF
:1088B000019400F021F800F023FEC04618020020C9
:1088C00081A2000098AC0000A5AC0000084B10B5D8
:1088D0000400002B02D0002100E000BF054B186807
:1088E000836A002B00D09847200001F0F3FAC046BD
:1088F00000000000D8AC00000EB403B5010003ABCB
:10890000044804CB0068019300F016F902B008BCDB
:1089100003B01847180200200E4B70B500251E004A
:108920000D4CE41AA410A54204D0AB00F3589847AC
:108930000135F8E701F0D0FA084B00251E00084C7D
:10894000E41AA410A54204D0AB00F35898470135AF
:10895000F8E770BD20020020200200202002002045
:108960003002002010B5034B0100186800F066F8D3
:1089700010BDC0461802002010B5034B0100186856
:1089800000F016F810BDC04618020020002310B5F4
:108990009A4203D0CC5CC4540133F9E710BD030004
:1089A0008218934202D019700133FAE77047000031
:1089B00030B500293ED004390B68002B00DAC91805
:1089C0001D4A13681400002B02D14B60116031E086
:1089D0008B420DD90A688818834203D118685B68F6
:1089E00082180A604B60216024E08A4203D8130099
:1089F0005A68002AF9D11D685C198C420BD10968AC
:108A0000691858181960824214D1106852684118C8
:108A100019605A600EE08C4202D90C23036009E011
:108A200008680C18A24203D1146852682018086024
:108A30004A60596030BDC046F0110020032370B574
:108A4000CD1C9D43083506000C2D01D20C2505E0F8
:108A5000002D03DA0C230020336040E0A942F9D84E
:108A60001F4B1C681A002100002913D00B685B1BE8
:108A70000DD40B2B02D90B60CC181EE08C4202D116
:108A8000636813601AE04B6863600C0016E00C002A
:108A90004968E9E7134C2368002B03D1300000F04C
:108AA00033FB20602900300000F02EFB431CD1D0A6
:108AB0000323C41C9C43A0420AD125602000072246
:108AC0000B30231D9043C31A09D05A42E25006E0EE
:108AD000211A300000F018FB431CEED1BAE770BD3C
:108AE000F0110020EC110020936810B5013B936059
:108AF000002B05DA9469A34208DBCBB20A2B05D020
:108B00001368581C10601970C8B201E000F02CFC0A
:108B100010BDF8B506000F001400D518AC4208D0FF
:108B200021783A003000FFF7DFFF0134431CF5D114
:108B300000E00020F8BD0000F0B59FB006000F0077
:108B400002920593002804D08369002B01D100F024
:108B5000D3FD7F4B9F4201D1776808E07D4B9F4258
:108B600001D1B76803E07C4B9F4200D1F768BB8915
:108B70001B070AD53B69002B07D0002306AD6B61AC
:108B800020336B761033AB763DE03900300000F0D7
:108B900043FC0028F1D001204042D6E0059A111D87
:108BA00012680591002A00DA7FE0099201342378E7
:108BB0002E2B00D18DE021780322684800F082FE40
:108BC000002807D0654B2A68C01A4023834013430E
:108BD0002B6001342178631C0622614802932976B8
:108BE00000F070FE002800D19DE05E4B002B00D00D
:108BF00090E00722059B07339343083305936B6985
:108C0000039A9B186B61029C2378002B04D1029B72
:108C1000E31A049312D003E0252BF8D00134F3E7D4
:108C2000049B029A39003000FFF773FF431C00D108
:108C300086E06A69049B944663446B612378002B49
:108C40007ED00122002352426A6002A95432521897
:108C500001342B60EB60AB601370AB6521780522AB
:108C6000414800F02FFE002808D03F4B2A68C01A68
:108C70000123834013432B600134EFE72B68DA06AE
:108C800004D55322202102A8121811701A0704D506
:108C900053222B2102A81218117022782A2A00D1FF
:108CA0007CE7099B00200A2105E05242EA6002228B
:108CB00013432B607AE72278303A092A04D84B43D1
:108CC00001349B180120F6E7002800D16FE70993D3
:108CD0006DE763782A2B0AD1059B02341A1D1B68A5
:108CE0000592002B01DA01235B42079363E700231F
:108CF0000A201A0001346B6021783039092904D820
:108D00004243013452180123F6E7002B00D152E709
:108D1000079250E705AB00933A00144B290030004E
:108D200000E000BF07E005AB00933A000F4B2900BD
:108D3000300000F08BF80390039B013300D05EE716
:108D4000BB895B0600D526E70B981FB0F0BDC04677
:108D500010AE000030AE000050AE0000E2AC0000EB
:108D6000E6AC000000000000DCAC0000138B00004B
:108D7000F7B5170001938A680B6900900C009342C5
:108D800000DA130022003B6043321278002A01D03F
:108D900001333B6023689B0602D53B6802333B608E
:108DA000062523681D401ED0230043331B785A1E1E
:108DB0009341226892061CD53020E1184331087097
:108DC00021005A1C45310978A21843320233117030
:108DD0000FE022000123193201990098089EB04744
:108DE000431C0ED00135E3683A689B1A9D42F0DBC4
:108DF000DAE72200019943320098089DA847431CF6
:108E000002D10120404220E006232068E1683A6850
:108E100003400025042B03D18D1AEB43DB171D40C3
:108E2000A3682269934201DD9B1AED180027BD4219
:108E30000AD0220001231A3201990098089EB047F7
:108E4000431CDED00137F2E70020FEBDF0B58BB049
:108E500006920A0043320793059004920A7E0C00A2
:108E6000109B6E2A00D1ABE011D8632A22D009D81A
:108E7000002A00D1B5E0582A00D0C5E045310A707B
:108E8000814A4FE0642A1DD0692A1BD0BCE0732AB6
:108E900000D1AAE009D86F2A29D0702A00D0B3E007
:108EA000202209680A43226037E0752A1FD0782AF9
:108EB00033D0A9E00E001A684236111D19601368FC
:108EC0003370A4E021681A68080606D4490604D560
:108ED000111D19600023D55E02E0111D196015688F
:108EE000002D3BDA2D23049A6D42137036E0216881
:108EF0001A68080606D4490604D51568111D1960BC
:108F0000ADB202E0111D196015685F4B227E03931C
:108F100008276F2A1DD00A271BE02200782145323E
:108F200011705A4A19680392081D226818600D686A
:108F3000100602D4500600D5ADB2D30702D52023C7
:108F40001A4322601027002D03D1202322689A4360
:108F500022602300002243331A7002E00A274A4BA2
:108F600003936368A360002B09DB0422216891430B
:108F70002160002D05D1049E002B11D07BE0002D37
:108F800079D0049E28003900FDF7CAFE039B013EFC
:108F90005B5C280033703900FDF73CFE051EF1D103
:108FA000082F09D12368DB0706D56368226993423D
:108FB00002DC3023013E3370049B9B1B23612BE0BA
:108FC00009681A68080607D4490605D5111D1960F5
:108FD0001368A28A1A8004E0111D1960136862697F
:108FE0001A600023049E236116E01A68111D19609F
:108FF000166800216268300000F064FC002801D08F
:10900000801B6060636803E02600423632700123F3
:1090100023610023049A1370079B09AA009321007F
:10902000069B0598FFF7A4FE431C02D10120404295
:1090300027E02369320006990598079DA847431C3D
:10904000F4D0236800259B070FD4099BE068984261
:1090500017DA180015E02200012319320699059845
:10906000079EB047431CE1D00135E368099A9B1A7B
:109070009D42F0DBE9E72600039B42361B78337004
:109080008EE70BB0F0BDC046EDAC0000FEAC0000BA
:10909000154B10B51C68A36B002B15D11820FFF7DA
:1090A00061FC124BA0630380114B01224380114BE2
:1090B0008380114BC380114B038105234381063309
:1090C0008381002302614361A46B0D4A20696169B9
:1090D0000C4BFDF761FF01220023801859412061EC
:1090E00061614800400810BD180200200E330000E6
:1090F000CDABFFFF341200006DE6FFFFECDEFFFF9B
:109100002D7F954C2DF45158002370B5064C050069
:109110000800236000F0C8FE431C03D12368002B25
:1091200000D02B6070BDC046DC2400200CB430B5EC
:10913000164B9DB00C1E1D6804DA8B2301202B609A
:1091400040421DE0822302A99B008B8100230290F4
:1091500008619C4200D0631E8B604B6101235B421F
:10916000CB81209A21AB2800019300F053FC431CD3
:1091700001DA8B232B60002C02D00023029A13709B
:109180001DB030BC08BC02B01847C0461802002011
:109190000EB410B59DB002A9029008610B4882245C
:1091A00088604861012040421FABC881084804CB59
:1091B000A400006801938C8100F02CFC0023029A2B
:1091C00013701DB010BC08BC03B01847FFFFFF7F31
:1091D0001802002002780B78002A03D001300131F8
:1091E0009A42F7D0D01A7047031C0A7801311A70DE
:1091F0000133002AF9D170470023C25C0133002AF1
:10920000FBD1581E7047030030B5002A0DD00C78F2
:1092100001335D1E013A2C700131002CF5D19A18F2
:109220009A4202D01C700133FAE730BDF0B51E003F
:10923000454B87B01B680192029308220B000590F2
:1092400003911C7802995D1C09194878104001D0DF
:109250002B00F6E72D2C04D19D1C5C780123009394
:1092600004E000902B2C01D15C789D1C002E02D0D4
:10927000102E0AD162E0302C5ED120222B7893434D
:10928000582B54D110266C780235009F31007B1E7C
:109290009F412E4BFF183800FDF742FD3800049126
:1092A0003100FDF7B7FC00230322070094461800A5
:1092B000029A121951780422114201D0303C07E081
:1092C0006246114017D03722012900D02032A41A5B
:1092D000A64210DD5A1C0BD0B84207D802D1049B1D
:1092E0009C4203DC70430123201801E001235B4210
:1092F0002C780135DCE75A1C0BD10098059A431EE7
:109300009841124BC01822231360019B002B0AD1F5
:1093100017E0009A002A00D04042019A002A10D09B
:10932000039A002B00D06A1E019B1A6009E03024CA
:10933000002EAAD10826A8E70A26A6E7302C9CD042
:10934000A3E707B0F0BDC0461C020020FFFFFF7F6F
:1093500010B513000A00010002480068FFF766FF1D
:1093600010BDC04618020020F8B505000F0014001B
:10937000002804D08369002B01D100F0BDF9234BF4
:109380009C4201D16C6808E0214B9C4201D1AC6841
:1093900003E0204B9C4200D1EC68A369A360A38941
:1093A0001B070AD52369002B07D023682269FEB268
:1093B000981A636998420FDB08E02100280000F04A
:1093C0002BF80028F1D0012040421DE021002800A8
:1093D00000F024F90028F6D1A3680130013BA36016
:1093E00023685A1C22601F706369984205D0A389C4
:1093F0003000DB0708D50A2E06D12100280000F036
:109400000DF90028DFD13000F8BDC04610AE0000D5
:1094100030AE000050AE0000354B70B51D68060040
:109420000C00002D05D0AB69002B02D1280000F004
:1094300063F9304B9C4201D16C6808E02E4B9C4292
:1094400001D1AC6803E02D4B9C4200D1EC68A389AC
:109450009AB2110723D4D10607D409220120326021
:1094600037321343A381404240E0530713D5616B69
:10947000002908D023004433994202D03000FFF77E
:1094800097FA002363632422A3899343A3810023D3
:109490006360236923600822A3891343A38123699E
:1094A000002B0BD1A023A2899B00134080229200A5
:1094B000934203D02100300000F0B2F90123A289C9
:1094C000134005D00023A36063695B42A36103E0FE
:1094D000910700D46369A36000202369834205D10A
:1094E000130603D540231A43A281013870BDC0463C
:1094F0001802002010AE000030AE000050AE000098
:1095000010B5062000F0AEFB012000F0E3FC0000E7
:10951000F7B58A8905000C0013075AD44B68002B55
:1095200002DC0B6C002B19DDE76A002F16D000233C
:109530002E682B6080235B011A4001D0606D14E01F
:109540000123216A2800B847431C0ED12B68002B49
:109550000BD01D2B01D0162B02D12E6000205AE01B
:109560004022A3891343A38155E0A3895B0706D555
:109570006368C01A636B002B01D0236CC01A0023F0
:109580000200216A2800E76AB847A389421C06D175
:1095900029681D293AD8204ACA40D20736D5002268
:1095A000626022692260DB0405D5431C02D12B686E
:1095B000002B00D16065616B2E600029CED02300A6
:1095C0004433994202D02800FFF7F2F9002060638B
:1095D00021E00F69002FC1D00B680F60DB1B0193E6
:1095E0000023920700D14B69A36003E0019B3F1861
:1095F0001B1A0193019B002BB0DD019B3A00216AED
:109600002800A66AB0470028F0DCA3894022012088
:109610001343A3814042FEBD010040200B6970B599
:1096200005000C00002B01D100201CE0002804D014
:109630008369002B01D100F05FF80B4B9C4201D1F4
:109640006C6808E0094B9C4201D1AC6803E0084B10
:109650009C4200D1EC680C22A35E002BE4D02100D8
:109660002800FFF755FF70BD10AE000030AE0000BF
:1096700050AE000010B5024900F0B0F810BDC04671
:109680001D960000002310B5040003604360836052
:1096900081814366C28103614361836119000822AD
:1096A0005C30FFF77CF9054B24626362044BA362D4
:1096B000044BE362044B236310BDC046A59C00002D
:1096C000CD9C0000059D0000319D000070B568250F
:1096D0004B1E5D430E0029007431FFF7AFF9041EE5
:1096E00008D000212A00016046600C30A06068327A
:1096F000FFF755F9200070BD836913B50400002BF6
:1097000028D18364C3640365134B144A1B688262C7
:109710000193984201D101238361200000F020F8D9
:109720006060200000F01CF8A060200000F018F835
:109730000022E06004216068FFF7A4FF01220921F4
:10974000A068FFF79FFF02221221E068FFF79AFF4F
:109750000123A36113BDC046D8AC0000759600007C
:10976000F8B51D4B06001D68AB69002B02D128001F
:10977000FFF7C2FF4835AC686B68013B05D40C228B
:10978000A75E002F10D06834F7E72B68002B01D0BC
:109790002D68F0E704213000FFF798FF28600028CB
:1097A000F6D10C23336016E0012320005B42E381F5
:1097B0000233A38167662760A760676027616761DE
:1097C000A7615C3008223900FFF7E9F820006763E1
:1097D000A763A764E764F8BDD8AC0000F7B5040040
:1097E0000700002601914834002C16D06368A56854
:1097F0000093009B013B00930DD4AB89012B08D94A
:109800000E22AB5E013304D029003800019B98473B
:1098100006436835EDE72468E6E73000FEBD00004A
:10982000F0B58B8991B006000C009B0726D40E235F
:10983000C95E002904DA8023A5891D4010D10CE0FF
:1098400001AA00F0A1FA0028F5DBF023029D1B021B
:109850001D401A4BED186B425D418027FF0001E06F
:109860000025402739003000FFF7E8F800280CD128
:10987000A3899A051FD402221343A38123004733EF
:10988000236023610123636115E080220C4BB362E6
:10989000A38920601343A38120616761002D0AD052
:1098A0000E23E15E300000F081FA002803D001228F
:1098B000A3891343A38111B0F0BDC04600E0FFFFB0
:1098C00075960000C9B28218904204D003788B428A
:1098D00002D00130F8E70020704710B5884202D965
:1098E0008B18984201D3002305E09B1A013A08D354
:1098F000995C8154FAE7934203D0CC5CC4540133A1
:10990000F9E710BDF8B506000C001500002904D1D8
:109910001100FFF793F8040018E0002A03D1FFF7C5
:1099200047F82C0012E000F067FA85420ED92900B2
:109930003000FFF783F8071E07D021002A00FFF749
:1099400025F821003000FFF733F83C002000F8BD77
:10995000F0B58E6885B007000C00039201939E421B
:1099600043D890238A89DB001A423ED00325096937
:10997000236801985B1A029363695D43EB0F5D19DD
:10998000029B6D1001331B18AB4200D91D0053051B
:1099900010D529003800FFF751F8061E14D0029A9E
:1099A0002169FEF7F3FFA289194B1340802213436C
:1099B000A38112E02A003800FFF7A4FF061E0CD195
:1099C00021693800FEF7F4FF0C23402201203B60A0
:1099D000A38940421343A38117E0029B2661F61836
:1099E00026606561019EED1AA560019BB34200D21D
:1099F0001E00320003992068FFF76FFF0020A36864
:109A00009B1BA36023689E19266005B0F0BDC0466D
:109A10007FFBFFFFF0B59FB0029005938B890F008D
:109A200016001B0610D50B69002B0DD14021FFF746
:109A300005F838603861002804D10C23029A0138F7
:109A40001360D8E040237B61002306AD6B612033B7
:109A50006B761033AB7634002378002B03D1A31B35
:109A6000049312D003E0252BF9D00134F4E7A31BB3
:109A7000320039000298FFF76BFF431C00D1B4E0BD
:109A80006A69049B944663446B612378002B00D180
:109A9000ABE00122002352426A6002A954325218FC
:109AA00001342B60EB60AB601370AB65534E2178D3
:109AB00005223000FFF706FF002807D00123801B96
:109AC00083402A68013413432B60EFE72B68DA06E2
:109AD00004D55322202102A8121811701A0704D5A8
:109AE00053222B2102A81218117022782A2A03D09F
:109AF000099B00200A210EE0059A111D12680591AC
:109B0000002A01DB099204E05242EA600222134378
:109B10002B6001340BE02278303A092A04D84B43F9
:109B200001349B180120F6E7002800D00993237820
:109B30002E2B1ED163782A2B0AD1059B02341A1DC5
:109B40001B680592002B01DA01235B42079310E0AA
:109B500000230A201A0001346B602178303909296A
:109B600004D84243013452180123F6E7002B00D0F9
:109B70000792234E217803223000FFF7A3FE00282E
:109B800006D04023801B83402A68013413432B6096
:109B9000217806221B48661C2976FFF793FE0028D1
:109BA00012D0194B002B06D10722059B0733934394
:109BB0000833059314E005AB00933A00134B2900DA
:109BC000029800E000BF07E005AB00933A000F4B9E
:109BD00029000298FFF73AF90390039B013304D060
:109BE0006B69039A9B186B6135E7BB890B985B0621
:109BF00001D5012040421FB0F0BDC046DCAC0000E2
:109C0000E2AC0000E6AC000000000000519900004A
:109C100070B504000D1E1F2D04D91623036001200A
:109C200040421EE0426C002A04D08B00D218136818
:109C3000002B08D1200000F031F82A00010020009C
:109C400000F01AF80DE00020012B0AD0591C03D1B6
:109C500017332360013004E0002428001460984783
:109C6000200070BD10B5034B01001868FFF7D0FF4E
:109C700010BDC04618020020002370B5064C050038
:109C800008001100236000F0F7F8431C03D123689B
:109C9000002B00D02B6070BDDC24002010B500F03C
:109CA000DBF810BD70B50C000E25495F00F0B0F870
:109CB000002803DB636D1B18636503E0A289024B78
:109CC0001340A38170BDC046FFEFFFFFF8B51F0032
:109CD0008B8905000C001600DB0505D50E23C95E37
:109CE0000022022300F074F8A289054B28001340DB
:109CF000A38132000E23E15E3B0000F01FF8F8BDA7
:109D0000FFEFFFFF70B50C000E25495F00F060F813
:109D1000A389421C03D1054A1340A38104E0802299
:109D200052011343A381606570BDC046FFEFFFFF82
:109D300010B50E23C95E00F015F810BD70B5050012
:109D4000080011000022064C22601A0000F0BAF848
:109D5000431C03D12368002B00D02B6070BDC0468C
:109D6000DC240020002370B5064C050008002360A9
:109D700000F062F8431C03D12368002B00D02B6055
:109D800070BDC046DC240020002370B5064C0500E1
:109D900008001100236000F057F8431C03D123682A
:109DA000002B00D02B6070BDDC240020002370B598
:109DB000064C05000800236000F056F8431C03D150
:109DC0002368002B00D02B6070BDC046DC2400202F
:109DD00070B50500080011000022064C22601A0030
:109DE00000F052F8431C03D12368002B00D02B60F5
:109DF00070BDC046DC2400200B1F1A68101F002A0B
:109E000004DA891804390B68D01804387047000048
:109E100070B50500080011000022064C22601A00EF
:109E200000F03AF8431C03D12368002B00D02B60CC
:109E300070BDC046DC24002058220120014B404266
:109E40001A607047DC24002058220120014B404258
:109E50001A607047DC24002058220120014B404248
:109E60001A607047DC2400205822024B00201A6040
:109E70007047C046DC24002058220120014B40429C
:109E80001A607047DC24002058220120014B404218
:109E90001A607047DC24002058220120014B404208
:109EA0001A607047DC240020044A1368002B03D09A
:109EB0001818106018007047014BF9E7F4110020E2
:109EC000E024002058220120014B40421A607047D4
:109ED000DC240020FEE7C046F8B5C046F8BC08BC4C
:109EE0009E467047F8B5C046F8BC08BC9E46704711
:109EF000F40600008A06000006070000360700008E
:109F00006E070000A2070000DA0700000208000048
:109F10004608000088080000E0080000260900004C
:109F200094090000DC090000040A0000420A000055
:109F30008C0A0000B60A0000F20A00002E0B000096
:109F40006A0B0000F00B0000BA0C0000480D000086
:109F5000A40D0000E60D0000080E0000100E000029
:109F6000F20E0000F4060000F4060000F406000003
:109F7000F4060000400F0000AA0F000014100000BB
:109F80005E100000C010000046110000CE1100005D
:109F90001C12000066120000AC120000F812000053
:109FA0004413000090130000DE1300002C14000086
:109FB0006A140000E0140000101500005C15000099
:109FC000A8150000F41500002E1600007A160000F7
:109FD000C6160000F4060000F4060000F4060000B7
:109FE0002E1700005E1700008E170000BA17000041
:109FF000EA17000016180000F4060000F40600003E
:10A00000F4060000F406000046180000881800005E
:10A01000D818000008190000341900006019000069
:10A02000AA190000F4060000F4060000F40600007F
:10A03000D8190000081A0000381A0000681A000039
:10A04000941A0000C41A0000F01A00001A1B000045
:10A05000441B0000741B0000A41B0000D01B000068
:10A06000FC1B00002C1C0000581C0000F406000023
:10A07000F4060000F4060000F4060000F4060000F8
:10A080009C1C0000C81C0000F41C0000201D0000E7
:10A090004C1D0000841D0000BC1D0000F41D0000CC
:10A0A0002C1E0000581E0000861E0000B61E000078
:10A0B000F4060000F4060000F4060000F4060000B8
:10A0C000F4060000F4060000F4060000F4060000A8
:10A0D000F4060000F4060000F4060000F406000098
:10A0E000F4060000F4060000E41E0000121F000049
:10A0F00066616C73650074727565006C69737420B9
:10A100006F66202564206974656D73006F626A65EF
:10A110006374206F6620636C6173733A202564005A
:10A12000537461636B20756E646572666C6F770043
:10A130000D0A564D2050616E69633A2025730D0A51
:10A1400000496E73756666696369656E74206D6536
:10A150006D6F727920666F72204D6963726F426C09
:10A160006F636B73206F626A6563742068656170EA
:10A1700000496E73756666696369656E74206D6506
:10A180006D6F727920666F72204D6963726F426CD9
:10A190006F636B7320737461636B00626164206F23
:10A1A000626A65637420617420256C640A002578F6
:10A1B0003A20256420776F7264732C20636C61737E
:10A1C0007349442025640A004865616465723A2039
:10A1D00025780A0009307825782C0A006D697363A8
:10A1E0000073696E002564202564202564202564A1
:10A1F0000A00426164207265636F726420666F7545
:10A200006E6420647572696E6720696E6974696135
:10A210006C697A6174696F6E210A004E6F742065F3
:10A220006E6F75676820726F6F6D206576656E2042
:10A23000616674657220636F6D70616374696F6EBF
:10A240000A00526573746F72696E6720256420730B
:10A250006372697074732E2E2E005374617274656C
:10A2600064002D2D2D2D2D0A0050657273697374B5
:10A27000656E74204D656D6F727920546573740A34
:10A280000A000A496E697469616C697A696E6720AF
:10A290004D656D6F72790A004D656D6F7279206939
:10A2A0006E74697469616C697A65643B2077726960
:10A2B00074696E67207265636F7264732E2E2E0A46
:10A2C000005265636F7264206174206F6666736507
:10A2D000742025643A2025642025642025642025E7
:10A2E000642028256420776F726473290A00466908
:10A2F0006E616C3A2063757272656E7420256420FD
:10A3000075736564202564206330202564206331E3
:10A310002025640A00E2ECF0F4F8FC00046E756D90
:10A32000626572006E6F6E65006F746865720070B2
:10A3300061697200737472696E6700726164696F3B
:10A340000064697361626C65526164696F006D6578
:10A3500073736167655265636569766564007061F2
:10A36000636B657452656365697665007061636BE4
:10A37000657453656E6400726563656976656449EA
:10A380006E74656765720072656365697665644DB4
:10A39000657373616765547970650072656365699B
:10A3A000766564537472696E670073656E64496E96
:10A3B00074656765720073656E64506169720073DD
:10A3C000656E64537472696E670073657443686187
:10A3D0006E6E656C0073657447726F75700073659F
:10A3E00074506F776572007369676E616C53747235
:10A3F000656E677468004E6F2066726565207461D3
:10A40000736B20656E74726965730057656C636F5A
:10A410006D6520746F204D6963726F426C6F636B62
:10A420007321004D656D6F727920636C6561726593
:10A43000642E00416C6C207461736B732073746FB5
:10A4400070706564007630353600202573202573E2
:10A450000000000007000000030000006D69637247
:10A460006F3A62697400686173546F6E6500706C56
:10A470006179546F6E6500686173536572766F0021
:10A48000736574536572766F000000000000000071
:10A4900001000000020000000300000004000000B2
:10A4A0000A0000006E6574006861735769466900B0
:10A4B0007374617274576946690073746F70576979
:10A4C00046690077696669537461747573006D79C4
:10A4D000495041646472657373007468696E6744BF
:10A4E00065736372697074696F6E00636C65617225
:10A4F0005468696E674465736372697074696F6EDE
:10A5000000617070656E64546F5468696E6744656D
:10A51000736372697074696F6E001A1B1C03040602
:10A5200007090A1718191A1B1C03040607090A173A
:10A530001819646973706C6179006C696768744C90
:10A540006576656C0000000000000000010000005E
:10A5500002000000030000000400000005000000ED
:10A5600006000000070000000800000009000000CD
:10A570000A0000000B0000000C0000000D000000AD
:10A580000E0000000F00000010000000120000008C
:10A590001400000016000000180000001A0000005F
:10A5A0001C0000001E00000020000000230000002E
:10A5B00026000000290000002C0000002F000000F1
:10A5C00032000000360000003A0000003E000000AB
:10A5D00042000000460000004B0000005000000058
:10A5E000550000005A0000006100000068000000F3
:10A5F0006F000000760000007D0000008400000075
:10A600008B0000009200000099000000A0000000F4
:10A61000A7000000AE000000B5000000BC00000074
:10A62000C3000000CA000000D1000000D8000000F4
:10A63000DF000000E6000000ED000000F400000074
:10A64000FB000000FF0000000000000000080808F8
:10A6500000080A4A4000000A5FEA5FEA0ED92ED3DA
:10A660006E19324489330C924C924D080800000058
:10A6700004880808040804848488000A448A400086
:10A68000048EC480000000048800000EC00000009A
:10A6900000080001224488100C9252524C048C8411
:10A6A000848E1C824C901E1EC244924C06CA525F7D
:10A6B000E21FF01EC13E02448ED12E1FE2448810DC
:10A6C0000ED12ED12E0ED12EC48800080008000015
:10A6D000048004880244880482000EC00EC008046E
:10A6E0008244880ED126C0040ED135B36C0C925E24
:10A6F000D2521C925C925C0ED010100E1C925252E0
:10A700005C1ED01C901E1ED01C90100ED013712EFB
:10A7100012525ED2521C8808081C1FE242524C1290
:10A7200054981492101010101E113B75B13111394C
:10A7300035B3710C9252524C1C925C90100C925298
:10A740004C861C925C92510ED00C825C1FE4848477
:10A7500084125252524C1131312A44113135BB719D
:10A7600012524C9252112A4484841EC488101E0E28
:10A77000C808080E10080482410EC242424E048AE4
:10A78000400000000000001F0804800000000ED2FE
:10A79000524F10101C925C000ED0100E02424ED28E
:10A7A0004E0C925C900E06C81C88080ED24EC24C0D
:10A7B00010101C92520800080808024002424C1077
:10A7C000149814920808080806001B75B131001C83
:10A7D000925252000C92524C001C925C90000ED28D
:10A7E0004EC2000ED010100006C8049808080EC80B
:10A7F00007001252524F0011312A4400113135BB6B
:10A8000000124C8C9200112A4498001EC4881E0627
:10A81000C48C8486080808080818080C88180000EA
:10A820000C836073656E736F72730074656D706511
:10A830007261747572650074696C74580074696C27
:10A8400074590074696C745A00746F75636852654A
:10A8500061640069326352656164006932635772F2
:10A860006974650074667400656E61626C65446944
:10A8700073706C617900736574506978656C006CF5
:10A88000696E65007265637400726F756E646564ED
:10A890005265637400636972636C65007472696108
:10A8A0006E676C65007465787400535049436C6141
:10A8B00073733A3A535049436C617373284E52464E
:10A8C0005F5350495F547970652A2C2075696E7406
:10A8D000385F742C2075696E74385F742C2075692C
:10A8E0006E74385F742900705F73706920213D2099
:10A8F0004E554C4C002F55736572732F6A6F686EFE
:10A900006D616C6F6E65792F4C6962726172792F1F
:10A9100041726475696E6F31352F7061636B616769
:10A9200065732F73616E646565706D697374727998
:10A930002F68617264776172652F6E5246352F30D1
:10A940002E362E302F6C69627261726965732F53D7
:10A9500050492F5350492E637070000000000000D2
:10A9600000000000C34B0000894B0000AF4B00000B
:10A97000B94B0000E94B0000AD4B000003000000A4
:10A9800002000000010000000400000005000000BB
:10A99000110000000C0000000B000000120000007D
:10A9A0000A000000060000001A0000001400000069
:10A9B0001700000016000000150000001000000045
:10A9C000FFFFFFFFFFFFFFFF000000001E00000071
:10A9D0001900000018000000070000000800000037
:10A9E000090000000D0000000E0000000F00000034
:10A9F0001C0000001B0000001D00000013000000F0
:10AA0000000000000000304300000000000030C3E0
:10AA1000FB21F93FFB2109407CD91240FB21194061
:10AA20007A6A1F407CD92240BBFD2540FB2129408A
:10AA30003A462C407A6A2F405C4731407CD93240FC
:10AA40009C6B3440BBFD3540DB8F3740FB213940E8
:10AA50001BB43A403A463C405AD83D407A6A3F409F
:10AA60004C7E40405C4741406C1042407CD94240A3
:10AA70008CA243409C6B4440AC344540BBFD4540F8
:10AA8000CBC64640DB8F4740EB584840FB2149404E
:10AA900083F9A200444E6E00FC291500D15727000F
:10AAA000DD34F50062DBC0003C9995004190430025
:10AAB0006351FE00BBDEAB00B761C5003A6E2400F7
:10AAC000D24D42004906E00009EA2E001C92D10056
:10AAD000EB1DFE0029B11C00E83EA700F535820001
:10AAE00044BB2E009CE98400B4267000417E5F00C8
:10AAF000D6913900538339009CF439008B5F840070
:10AB000028F9BD00F81F3B00DEFF97000F980500F5
:10AB1000112FEF000A5A8B006D1F6D00CF7E36009B
:10AB200009CB2700464FB7009E663F002DEA5F0025
:10AB3000BA277500E5EBC7003D7BF100F739070048
:10AB400092528A00FB6BEA001FB15F00085D8D0026
:10AB5000300356007BFC4600F0AB6B0020BCCF00FE
:10AB600036F49A00E3A91D005E619100081BE6001F
:10AB700085996500A0145F008D40680080D8FF00B3
:10AB800027734D0006063100CA561500C9A8730088
:10AB90007BE260006B8CC00002000000030000003C
:10ABA000040000000600000000000040FB21F93F07
:10ABB000000000002D44743E000000809846F83CE0
:10ABC0000000006051CC783B00000080831BF0390E
:10ABD0000000004020257A38000000802282E33601
:10ABE000000000001DF369350000000000000000B7
:10ABF000056800002567000075680000896800008E
:10AC00007F68000003680000F76700009568000097
:10AC100021680000F36700000C7100006A700000FA
:10AC20006A70000068700000FE700000FE70000096
:10AC3000F470000068700000FE700000F470000006
:10AC4000FE700000687000000471000004710000D4
:10AC5000047100008E7100000C7D0000CC7B0000B0
:10AC6000CC7B0000CA7B0000E47C0000E47C000098
:10AC7000D67C0000CA7B0000E47C0000D67C00008B
:10AC8000E47C0000CA7B0000EC7C0000EC7C00004F
:10AC9000EC7C0000EC7E00002C2066756E6374690D
:10ACA0006F6E3A2000617373657274696F6E202253
:10ACB000257322206661696C65643A2066696C655B
:10ACC00020222573222C206C696E65202564257353
:10ACD00025730A0043000000B8010020232D302B0B
:10ACE0002000686C4C00656667454647003031328D
:10ACF00033343536373839414243444546003031E4
:10AD00003233343536373839616263646566000042
:10AD1000202020202020202020282828282820200B
:10AD20002020202020202020202020202020202023
:10AD3000881010101010101010101010101010109B
:10AD4000040404040404040404041010101010107B
:10AD50001041414141414101010101010101010154
:10AD60000101010101010101010101101010101088
:10AD70001042424242424202020202020202020225
:10AD8000020202020202020202020210101010204D
:10AD900000000000000000000000000000000000B3
:10ADA00000000000000000000000000000000000A3
:10ADB0000000000000000000000000000000000093
:10ADC0000000000000000000000000000000000083
:10ADD0000000000000000000000000000000000073
:10ADE0000000000000000000000000000000000063
:10ADF0000000000000000000000000000000000053
:10AE00000000000000000000000000000000000042
:10AE10000000000000000000000000000000000032
:10AE20000000000000000000000000000000000022
:10AE30000000000000000000000000000000000012
:10AE40000000000000000000000000000000000002
:10AE500000000000000000000000000000000000F2
:10AE600000000000000000000000000000000000E2
:04AE700000000000DE
:08AE74000053FF7F0100000004
:10AE7C00FFFFFFFFE1A100004D21000041A30000F6
:10AE8C00212800004EA30000392B00005EA3000017
:10AE9C00D92A00006CA30000C52C000077A3000089
:10AEAC003D28000087A30000A52800009BA30000FC
:10AEBC004D280000AAA30000DF2D0000B6A300005F
:10AECC00692D0000BFA300000F2D0000CAA30000D5
:10AEDC00552A0000D5A30000DD290000DEA30000E8
:10AEEC00112A0000E7A300005528000019FCFFFF01
:10AEFC00FFFFFFFF66A40000613A00006EA4000093
:10AF0C005D3A000077A40000653A000080A40000C0
:10AF1C00693A0000A8A40000193D0000B0A400008C
:10AF2C003D3D0000BAA40000473D0000C3A4000052
:10AF3C00513D0000CEA400005B3D0000DAA40000EF
:10AF4C00273D0000EBA40000313D000001A50000EE
:10AF5C001D3D00003AA500007D3D000018000000DA
:10AF6C00FF0000002BA800008D45000037A8000052
:10AF7C00F94800003DA800000949000043A8000062
:10AF8C001949000049A80000C145000053A8000061
:10AF9C00294900005BA800000147000068A80000D8
:10AFAC00B549000076A80000B94900007FA8000050
:10AFBC00BD49000084A80000C149000089A8000018
:10AFCC00C549000095A80000C94900009CA80000D4
:10AFDC00B1490000A5A80000AD4900000300000025
:10AFEC0002000000080000000A000000FFFFFFFF45
:10AFFC000000000001000000000002000100000041
:10B00C00FFFFFFFF00000000020000000000040032
:10B01C0002000000FFFFFFFF000000000300000023
:10B02C0000000800030000000000000010AE00004B
:10B03C0030AE000050AE0000000000000000000028
:10B04C000000000000000000D4AC00000000000074
:10B05C0000000000000000000000000000000000E4
:10B06C0000000000000000000000000000000000D4
:10B07C0000000000000000000000000000000000C4
:10B08C000000000000000000B80100200FAD00001F
:10B09C0039010000594B0000794E0000F96A00009C
:08B0AC000D010000000000008E
:04000003000062B5E2
:00000001FF
